:100000000020001015010000D1000000D500000004
:1000100000000000000000000000000000000000E0
:10002000000000000000000000000000D9000000F7
:100030000000000000000000DD0000006D3700003F
:10004000E5000000E5000000E5000000E50000001C
:10005000E5000000E5000000E5000000E50000000C
:10006000E5000000E5000000E5000000E5000000FC
:100070000D280000E5000000B55D0000AD63000044
:100080006D640000E500000069680000E968000098
:10009000E5000000E5000000E5000000E5000000CC
:1000A00000000000E5000000E5000000E5000000A1
:1000B00000000000E500000045610000688A0000C3
:1000C000000000109004000090040010F0140000E4
:1000D000FEE7C046FEE7C046FEE7C046FEE7C04674
:1000E000FEE7C046FEE7C04610B5002304E0046802
:1000F0000C600433043004319342F8D310BDC04681
:100100000023002202E00260043304308B42FAD361
:100110007047C04638B5164B00221A60AA229A6072
:1001200055229A60134B144C07E0186859681D1C3F
:100130000C359A68FFF7D8FF2B1CA342F5D307E0D4
:1001400018681D1C08355968FFF7DAFF2B1C00E002
:100150000A4CA342F4D30A4B1B680A4A196811607F
:100160005A68094B1A6006F0BDFF07F063F9FEE715
:1001700000400040BC000000C8000000D0000000AB
:100180000000FC1F7C05001078050010FFFFFFFF3A
:10019000FFFFFFFFFFFFFFFFFFFFFFFFFFFFFFFF6F
:1001A000FFFFFFFFFFFFFFFFFFFFFFFFFFFFFFFF5F
:1001B000FFFFFFFFFFFFFFFFFFFFFFFFFFFFFFFF4F
:1001C000FFFFFFFFFFFFFFFFFFFFFFFFFFFFFFFF3F
:1001D000FFFFFFFFFFFFFFFFFFFFFFFFFFFFFFFF2F
:1001E000FFFFFFFFFFFFFFFFFFFFFFFFFFFFFFFF1F
:1001F000FFFFFFFFFFFFFFFFFFFFFFFFFFFFFFFF0F
:10020000FFFFFFFFFFFFFFFFFFFFFFFFFFFFFFFFFE
:10021000FFFFFFFFFFFFFFFFFFFFFFFFFFFFFFFFEE
:10022000FFFFFFFFFFFFFFFFFFFFFFFFFFFFFFFFDE
:10023000FFFFFFFFFFFFFFFFFFFFFFFFFFFFFFFFCE
:10024000FFFFFFFFFFFFFFFFFFFFFFFFFFFFFFFFBE
:10025000FFFFFFFFFFFFFFFFFFFFFFFFFFFFFFFFAE
:10026000FFFFFFFFFFFFFFFFFFFFFFFFFFFFFFFF9E
:10027000FFFFFFFFFFFFFFFFFFFFFFFFFFFFFFFF8E
:10028000FFFFFFFFFFFFFFFFFFFFFFFFFFFFFFFF7E
:10029000FFFFFFFFFFFFFFFFFFFFFFFFFFFFFFFF6E
:1002A000FFFFFFFFFFFFFFFFFFFFFFFFFFFFFFFF5E
:1002B000FFFFFFFFFFFFFFFFFFFFFFFFFFFFFFFF4E
:1002C000FFFFFFFFFFFFFFFFFFFFFFFFFFFFFFFF3E
:1002D000FFFFFFFFFFFFFFFFFFFFFFFFFFFFFFFF2E
:1002E000FFFFFFFFFFFFFFFFFFFFFFFFFFFFFFFF1E
:1002F000FFFFFFFFFFFFFFFFFFFFFFFFFFFFFFFF0E
:10030000054AD023D0588021C9000143D150D1588B
:1003100010208143D15070470040044008B50120AF
:100320000521012201F000FF01200521002201F03A
:100330003BFFFA20400005F097FF01200521012234
:1003400001F032FF01200521002201F0EDFE1E2008
:1003500005F08AFF0120052101F05EFF08BDC046BF
:1003600070B5061C01200521012201F0DDFE0120EF
:100370000521012201F018FF0025012424E0201CA2
:100380000521002201F010FF231C33400BD0062072
:1003900005F06AFF201C0521221C01F005FF5020FA
:1003A00005F062FF0AE0502005F05EFF201C0521E9
:1003B000221C01F0F9FE062005F056FF7608201CED
:1003C00005F052FF0135EDB2072DD8D901200521E6
:1003D000002201F0A9FE70BDF8B55F4656464D46B5
:1003E0004446F0B483468A46002291460027012401
:1003F00037E0D846C844424617703D1C261C2AE008
:10040000201C0521221C01F08FFE201C05213A1C16
:1004100001F0CAFE201C05F027FF201C0521221C2C
:1004200001F0C2FE201C05213A1C01F07DFE0220D5
:1004300005F01AFF201C052101F0EEFE002803D074
:1004400042461378334313702A2005F00DFF7600DF
:10045000F6B20135EDB2072DD2D94B460133DBB2EE
:100460009946D145C5D33CBC90469946A246AB4679
:10047000F8BDC04638B5011C164B8E229200985824
:100480001024A043985080229C588020C001204313
:1004900098500023104D002402E09A00545101337B
:1004A000072BFAD90D4AB423D0588724A043D05043
:1004B000D45803202043D050094B186807F0EBFBB9
:1004C0000138FF220240120201231A43054B1A6031
:1004D00038BDC04600800440800500100040044044
:1004E00088040010000002400023072282425B4182
:1004F0005B4218400E4B1A68FF218A431A60196844
:10050000012282400A43802149040A431A60094BB0
:10051000C21892001368002BFCDA054A10680649DD
:100520000140116000205A0001D41B04980D70474F
:100530000000024004800010FFFFFFF808B5012012
:100540000121012201F0F0FD0121C023014AD15017
:1005500008BDC0460040044008B5002807D000236D
:10056000074A1360074A1370074A137006E02F23E7
:10057000064AD25C0120012101F016FE08BDC046EA
:10058000980400109404001096040010E80B00106A
:1005900008B5614A136801331360604A926B934255
:1005A00007D92F235D4AD35C9A0702D501225C4B01
:1005B0001A702E23594AD35C002B00D1AAE0594B64
:1005C0001B68012B20D0002B05D0022B62D0032BFF
:1005D00000D185E09EE02F23504AD35CDA0705D591
:1005E00001200121012201F0DFFD04E001200121B1
:1005F000002201F0D9FD484B1B68052B00D889E08B
:100600000122484B1A6085E0444B1B6B834203DB9D
:10061000434B1B78002B39D0434A13780133DBB2AC
:100620001370032B03D83E4B1B78002B72D02F2363
:100630003A4AD35CDA0705D501200121002201F0F6
:10064000B3FD04E001200121012201F0ADFD2F23C3
:10065000324AD35C9A0708D50322324B1A603423FE
:100660002E4AD25C314B1A7054E000222E4B1A7085
:100670002A4B9A6B284B1B689A4203D20522294BBE
:100680001A6047E00222274B1A6043E00022264B03
:100690001A703FE0214B1B6B83421DDD224A137809
:1006A0000133DBB21370032B34D92F231B4AD35CE5
:1006B000DA0705D501200121012201F075FD04E0D2
:1006C00001200121002201F06FFD0022164B1A705B
:1006D0000122144B1A601DE00022134B1A7019E01E
:1006E000124A1378013BDBB21370002B12D10522A2
:1006F0000C4B1A602F23094AD35CDA0705D5012079
:100700000121012201F050FD04E00120012100221D
:1007100001F04AFD08BDC04690040010E80B00102F
:100720009504001098040010960400109404001022
:1007300008B5002802D0012805D009E000200C21CE
:1007400001F06AFD05E00220002101F065FD00E0F6
:10075000002043425841C0B208BDC0461D4B002294
:100760001A70E121490259605A701A7201215972B6
:100770003C20D8601A611975174898611748D861EC
:1007800020201A5421201A5459842421012058541D
:100790009621890199622C215A54114B1B78012B07
:1007A00003D902212C230B4AD1540A4B11212D22AB
:1007B000995400222E215A542F215A540949196361
:1007C000032034215854044999633C215A543D2153
:1007D0005A547047E80B001050460000A0800200F9
:1007E00004000010A086010008B5FFF7B7FF08BDA0
:1007F00004E00A7802701A1C01310130531E002AED
:10080000F7D17047C9B202E001701A1C0130531EC3
:10081000002AF9D17047C04670B5031C002001E0E2
:10082000291C331C541E002A07D05E1C18784D1C4E
:100830000B78C01A221C0028F2D070BD00E00130F5
:100840000378002B01D08B42F9D1181C7047C046A9
:10085000F8B55F4656464D464446F0B489460C68A6
:1008600000E0013423782F2BFBD05C2BF9D0866974
:10087000301C20210B22FFF7C5FF23782E2B1DD122
:10088000002100235A1CE35C2E2B05D1022A03D839
:100890007354131C0131F5E72F2B05D05C2B03D0CB
:1008A0000620202B00D99DE0A21849460A6020228C
:1008B000202B00D82422F272002093E0002700238E
:1008C000082290469B465A1C9246E55C202D58D93A
:1008D0002F2D56D05C2D54D02E2D01D047450DD351
:1008E0004346082B75D12E2D75D159468B00DBB2AE
:1008F0009B46534608270B229046E4E76BB2002B39
:1009000003DA0323594619438B462B1C7F33DBB292
:100910001E2B04D92B1C2033DBB21C2B14D85346BE
:1009200001335146625C111C40393E2903D94039DC
:10093000C9B27C2951D841460139B9424FD9791CF5
:10094000F55502377254BEE72948291CFFF776FF98
:10095000002846D12B1C413B192B04D802235A46B0
:100960001A43934609E02B1C613B192B05D8012340
:10097000594619438B46203DEDB2F5550137534694
:10098000A1E754444A46146000232022AA425B4156
:100990009B000620002F25D03278E52A01D10522C0
:1009A00032704146082903D159468A00D2B2934693
:1009B000032259460A40012A01D1102213430C2276
:1009C00059460A40042A01D108221343F372002039
:1009D00008E0062006E0062004E0062002E00620EB
:1009E00000E006203CBC90469946A246AB46F8BDC6
:1009F000147E0000F0B5474680B4041C0E1C056B45
:100A00008D4233D00379002B1FD03421091888463A
:100A100040782A1C012304F091F9031C0120002BCB
:100A200025D12371626A216A5318AB420DD9E77848
:100A300009E0226AAD18607841462A1C012304F0BF
:100A40007DF9013FFFB2012FF3D80020002E0ED018
:100A5000211C34316078321C012304F029F9031C75
:100A60000120002B03D12663002000E0002004BCFD
:100A70009046F0BD10B5041C0A1C011C34314078AE
:100A8000012304F015F90323002833D11A4BE15C4C
:100A900009021A4BE35C194309B20223184A914236
:100AA00028D16D23E25C12066C23E35C1B041A431D
:100AB0006B23E35C1B021A436A23E35C1A431202B2
:100AC000120A104B9A4214D08923E25C1206882342
:100AD000E35C1B0413438722A25C120213438622A9
:100AE000A25C13431B021B0A074A9B185A1E934120
:100AF00000E00023181C10BD330200003202000089
:100B000055AAFFFF46415400BABEABFF08B5031E0D
:100B10000DD002780920002A0CD0DA888A4209D147
:100B2000587804F005F8C30703D5032002E0092034
:100B300000E0002008BDC046F8B55F4656464D4669
:100B40004446F0B4161C03681C78303C092C05D8C8
:100B50005A783A2A02D10233036001E0C44B1C7870
:100B60000B20002C00D07CE1A300C24A9D580D60F0
:100B7000002D00D172E12B78002B0ED0687803F0A5
:100B8000D7FF031CD80708D40020002E00D168E14D
:100B90005B070A20DB17184063E100232B70E0B2EB
:100BA000687003F0EFFF031C0320D90700D558E15C
:100BB000002E03D00A205A0700D552E1281C00213C
:100BC000FFF758FF031C002401281BD1FB22520011
:100BD000AA5C002A16D0FE23FF33EC5C2406FE2319
:100BE0005B00EB5C1B041C43FC23FF33EB5C1B0230
:100BF0001C43FD235B00EB5C1C43281C211CFFF7FE
:100C000039FF031C032B00D12AE10D20002B00D05B
:100C100027E14023EA5C12023F23EB5C1A4312B245
:100C200080239B009A4200D01BE14B23EF5C3F02E4
:100C30004A23EB5C1F430DD15B23EF5C3F065A2335
:100C4000EB5C1B041F435923EB5C1B021F4358231F
:100C5000EB5C1F432F624423EB5CEB705A1E0D20AC
:100C6000012A00D9FDE07B439B464123E95CA97042
:100C7000002900D1F5E04B1E0B4200D0F1E04623E5
:100C8000EA5C12024523EB5C1A4390462A81120764
:100C900000D0E6E04823EA5C12024723EB5C1343F2
:100CA0000DD15723EA5C12065623EB5C1B041A4352
:100CB0005523EB5C1B021A435423EB5C1343432282
:100CC000A85C00024222AA5C104381460D204E46D9
:100CD000002E00D1C5E0321C5A4446463009121895
:100CE00092460D20934200D2BBE0981A06F0D3FF43
:100CF000031C0D20002B00D1B3E05F4E9E42B64195
:100D0000764201365D4A934200D903260233EB61F5
:100D100050462218EA62494662186A62032E15D1CB
:100D20000D204246002A00D09BE06322A95C090600
:100D30006222AA5C120411436122AA5C12021143CE
:100D40006022AA5C0A43AA629B0010E00D20414683
:100D5000002900D185E05A44AA62022E01D15B002D
:100D600005E003225A43520801210B40D318444A9C
:100D70009B185B0A0D209F4273D301235B422B61BA
:100D80000023EB60032E5DD16B716523EA5C1202D8
:100D90006423EB5C1A4312196A61291C34316878A8
:100DA000012303F085FF00284CD1364BEA5C120288
:100DB000354BEB5C1A4312B2344B9A4242D1372383
:100DC000EA5C12063623EB5C1B041A433523EB5C0A
:100DD0001B021A433423EB5C1A432D4B9A4231D148
:100DE0002C4BEA5C12062C4BEB5C1B041A432B4B7E
:100DF000EB5C1B021A4386239B00EB5C1A43284BD7
:100E00009A421FD1274BEA5C1206274BEB5C1B046E
:100E10001A43264BEB5C1B021A4388239B00EB5CB6
:100E20001343EB60224BEA5C1206224BEB5C1B0483
:100E30001A43214BEB5C1B021A4387239B00EB5C9C
:100E400013432B612E701D4A138801339BB213800C
:100E5000EB80002028632871A86102E00C2000E0EC
:100E600001203CBC90469946A246AB46F8BDC04620
:100E70009C040010A0040010F50F0000F5FF000016
:100E8000FF010000330200003202000055AAFFFFFC
:100E9000525261411B0200001A02000019020000B8
:100EA0007272416123020000220200002102000050
:100EB0001F0200001E0200001D0200009E04001020
:100EC000F8B5041C0021FFF795FD051E53D12378CA
:100ED000032B48D16379002B45D000262663271CBD
:100EE0003437381C002180229200FFF78BFC5522FA
:100EF000224BE254AA22224BE25452233422A3541E
:100F00003522A35461233622A3544122372162544F
:100F100072218620800021541A4821541A496254B3
:100F20001A4AA354236987229200A354190A184A23
:100F3000A154190C174AA1541B0E174AA354E36875
:100F400088229200A354190A144AA154190C144A75
:100F5000A1541B0E134AA3546078391C6269012303
:100F600003F0ECFE667160780021002203F036FF8A
:100F7000002800D00125281CF8BDC0463202000020
:100F800033020000190200001A0200001B020000D8
:100F90001D0200001E0200001F02000021020000CE
:100FA0002202000023020000031C0239C269023A37
:100FB00000208A4203D998784843DB6AC0187047FA
:100FC000F8B5051C0C1E012C61D90120EB698B4280
:100FD0006DD92B78022B28D0032B3BD0012B58D175
:100FE0004E088E19710A6B6A5918281CFFF702FD0A
:100FF000002851D1F305DB0DEB1830331F79013692
:10100000710A6B6A5918281CFFF7F4FC002846D1B6
:10101000F605F60DAD193035287900020743380979
:10102000E30744D43805000D41E0090A6B6A5918FA
:10103000281CFFF7DFFC002834D16400FF235B008D
:101040001C402B193433587800022C193034237982
:1010500018432CE0C9096B6A5918281CFFF7CAFC11
:10106000002822D1A400FE235B001C402B1934333E
:10107000D87800069A78120410435B781B02184354
:101080002C19303423791843000100090FE00120A6
:101090000DE0012040420AE00120404207E001202B
:1010A000404204E00120404201E001204042F8BDFE
:1010B00070B5041C0D1CE1808168022001293DD01F
:1010C0002368DA698A4239D9002903D11A78032AB8
:1010D00000D1996A002909D1E1601A890220AA4247
:1010E0002CD99A6A2B09D318236119E09E7836010E
:1010F0000DE02068FFF764FF011C431C19D0012894
:1011000019D92368DB69834217D9AD1BADB2B5424B
:10111000EFD2E1602068FFF747FF2B09C01820617C
:101120000F231D406B012268D31834336361002004
:1011300004E0012002E0022000E0022070BDC04671
:10114000F8B5051C0C1C161C0220012979D9EB6985
:101150008B4276D92B78022B41D0032B53D002201F
:10116000012B6CD14F08CF19790A6B6A5918281CCA
:10117000FFF740FC002862D1FB05DB0D0122144083
:101180000AD0EA1830321079FF21314009010F22CC
:1011900002400A43D2B200E0F2B2EB1830331A71C7
:1011A000013701232B71790A6B6A5918281CFFF744
:1011B00021FC002843D1FF05FF0D002C02D0360989
:1011C000F6B208E0EA19303211790F229143360560
:1011D000320F0E1C1643EF1930373E712FE0090A0B
:1011E0006B6A5918281CFFF705FC002827D16400FA
:1011F000FF22520014402A1934322C19303426713F
:10120000360A56701BE0C9096B6A5918281CFFF78B
:10121000F1FB002813D1A400FE22520014402A1929
:101220003432D1782C193034090909070E4326715C
:10123000310A5170310C9170360ED670FFE70122E1
:101240002A71F8BDF0B5474680B4051C88460029D0
:1012500006D1C668002E0ED0C269B2420DD90DE08B
:101260004146FFF7ADFE031E012B3FD9EA69464612
:101270009A4203D93FE0012600E00126341C0227F0
:101280000134EB69A34202D8012E31D93C1C281C41
:10129000211CFFF795FE002806D0421C2BD0012808
:1012A00029D0B442ECD125E0281C211C134AFFF7B9
:1012B00047FF002807D14346002B04D0281C414695
:1012C000221CFFF73DFF002808D1EC602B695A1C57
:1012D0000AD0013B2B6101236B7105E0441E604283
:1012E0004441644201231C43201C04E0012002E02D
:1012F000002000E0002004BC9046F0BDFFFFFF0F7F
:10130000F0B557464E464546E0B4041C0E1CC58851
:101310000135ADB20420002D75D02369002B72D0A9
:101320000F272F4064D101332361E168002904D1E4
:1013300022681389AB4266D95AE02B09206882786B
:10134000013A1A4254D1FFF73BFE80460220434641
:10135000012B58D9013353D02368DA69424540D86C
:101360000420002E4FD0181CE168FFF76BFF804669
:1013700007204346002B46D00220012B43D00120FA
:10138000013340D020680021FFF734FB031C01200B
:10139000002B38D120683430002180229200FFF7E2
:1013A00031FA2668301C4146FFF7FEFD3063002607
:1013B00001229246B1460DE052461A712068494614
:1013C000FFF718FB00281DD123681A6B01321A633E
:1013D0000136F6B223689A78B242EDD81A6B961BA2
:1013E0001E634346E36020684146FFF7DDFD206150
:1013F000E5807F012268D71934376761002002E059
:10140000012000E001201CBC90469946A246F0BD98
:1014100070B5041C0021FFF74BFE031C002B1CD1F0
:10142000082620682169FFF7E5FA051E14D16069D6
:101430000378002B0FD0C37A1E4205D1A1690B227D
:10144000FFF7EAF9002807D0201C0021FFF758FF1A
:10145000051EE6D000E00425281C70BDF0B583B061
:10146000041C01910B782F2B01D05C2B04D101318E
:1014700001910023A36002E003689B6983600199E6
:101480000B781F2B07D8201C0021FFF711FE051C2D
:101490000023636135E004261027201C01A9FFF713
:1014A000D7F9051E2DD1201CFFF7B2FFA169CA7A1A
:1014B00000280ED004281FD1910605D50023A36073
:1014C00063611642E9D01CE00525510719D5051CBA
:1014D00017E0164212D16369DA7A174210D05A7DAA
:1014E0001202197D0A431204D87E0002997E031C61
:1014F0000B431343A360D0E7051C02E0051C00E08A
:101500000525281C03B0F0BD70B5051C0021FFF7B0
:10151000CFFD041E11D128682969FFF76BFA041E5C
:101520000BD16A691378E52B07D0002B05D0281C56
:101530000121FFF7E5FE041EEDD0002C13D1286831
:101540002969FFF757FA041E0DD16E69301C00217E
:101550002022FFF757F9301CA9690B22FFF748F941
:101560002B6801221A71201C70BDC046F0B5474699
:1015700080B4041C0D1C0227012926D9C2698A42A5
:1015800023D900270123984618E0201C291CFFF7C7
:1015900017FD061E19D0012814D0421C14D0201C9F
:1015A000291C0022FFF7CCFD071E0ED123695A1C0F
:1015B00003D00133236143466371351CE269AA42BB
:1015C000E3D802E0022700E00127381C04BC904663
:1015D000F0BDC0460B2300280ED18300074A9B585C
:1015E000002B01D000221A70002901D000230B70BB
:1015F0008000024BC1500023181C7047A00400104B
:10160000F0B54F464646C0B48DB0061C0191171C7C
:10161000002303601F23134098461E223A4001A86E
:1016200005A9FFF789FA051C02AB0B93002804D12A
:1016300005A80199FFF712FF051C0A9C002D02D195
:10164000002C00D106251C233B424DD0002D0BD091
:10165000042D03D105A8FFF757FF051C08234246B8
:101660001A4390460A9C09E0E37A11221A4202D1F9
:101670007B0702D402E0072500E00825002D40D1B9
:10168000424612073DD502F0A9F8A073030AE3739E
:10169000030C2374000E60740023E37223776377D6
:1016A000A377E377627D1202217D0A431204E77E6D
:1016B0003F02A17E0F431743A376E376237563753C
:1016C000059801230371002F1BD0036B9946391C29
:1016D000FFF74CFF051E14D10598013FC76049462E
:1016E000FFF788F9051C0CE0002D0AD1E37ADA0631
:1016F00004D4BA0705D5DA0702D402E0042500E0D5
:101700000725002D0AD143461B0703D52023424657
:101710001A439046059B1B6BF3613462002D1ED16A
:101720004346B371627D1202217D0A431204E37EB7
:101730001B02A17E0B4313433361E27F1206A37F9A
:101740001B041343627F12021343227F1343F3608F
:101750000023B360B361059B3360DB88B380281C32
:101760000DB00CBC90469946F0BDC046F0B55F4642
:1017700056464D464446F0B483B0041C0F1C9046B8
:101780001E1C0023336081880068FFF7BFF9031E29
:1017900000D0C8E0A27951B20223002900DAC2E0E9
:1017A0000723D10700D4BEE0E268A368D51AA84594
:1017B00000D9B1E04546AFE0A368DA0500D08FE07C
:1017C0005A0A206881780139C9B20A40904619D175
:1017D000002B01D1206902E06169FFF7F1FB0128CC
:1017E00006D8A27980235B421343A37102239AE0B7
:1017F000411C06D1A27980235B421343A3710123CC
:1018000091E0606122689246101C6169FFF7CCFB91
:10181000002806D1A27980235B421343A3710223DF
:1018200081E08346C344690A89462DD042464A4432
:1018300051468B789A4202D942469A1A91465346AB
:1018400058784946CBB2391C5A4603F031FA002881
:1018500006D0A27980235B421343A371012362E087
:10186000A37940221A420BD0A1695A468B1A4B45E4
:1018700006D25B02F818019980229200FEF7B8FFA9
:101880004B465B0299463BE0A2695A4526D0A379B4
:101890004021194212D0534658780199012303F090
:1018A0004DFA002806D0A27980235B421343A3712E
:1018B000012338E0A37940218B43A371226850783B
:1018C00001995A46012303F0F3F9002806D0A279C2
:1018D00080235B421343A371012324E05B46A36191
:1018E000A268D105C90D80239B005B1A9946AB42C3
:1018F00000D9A94661182431381C4A46FEF778FF02
:101900004F44A1680B1C4B44A3603268131C4B442A
:1019100033604B46ED1A02E0211C24310191002D69
:1019200000D049E70023181C03B03CBC9046994600
:10193000A246AB46F0BDC046F8B55F4656464D469A
:101940004446F0B4041C0F1C151C1E1C00233360FD
:1019500081880068FFF7DAF8031E00D0E4E0A2797E
:1019600051B20223002900DADEE00723910700D4F8
:10197000DAE0E36859190022994252415242154077
:10198000C5E0A368DA0500D0A2E05A0A2068817891
:101990000139C9B20A40904624D1002B08D12369ED
:1019A000002B09D10021FFF74DFC031C206103E04F
:1019B0006169FFF747FC031C002B00D1AAE0012B53
:1019C00006D1A27980235B421343A3710223ABE0CB
:1019D0005A1C06D1A27980235B421343A3710123D1
:1019E000A2E06361A3794021194214D0211C243163
:1019F00022685078A269012303F0A0F9002806D0DC
:101A0000A27980235B421343A37101238CE0A37965
:101A100040218B43A37122689246101C6169FFF735
:101A2000C3FA002806D1A27980235B421343A37135
:101A3000022379E08346C344690A89462ED0424690
:101A40004A4451468B789A4202D942469A1A9146A4
:101A5000534658784946CBB2391C5A4603F06EF9C2
:101A6000002806D0A27980235B421343A37101238F
:101A70005AE0A2695946531A4B450BD2201C243018
:101A80005B02F91880229200FEF7B2FEA379402291
:101A90009343A3714B465B0299462DE0A1695945DA
:101AA00014D0A268E3689A4210D2211C2431524615
:101AB00050785A46012303F0FBF8002806D0A2799B
:101AC00080235B421343A37101232DE05B46A36196
:101AD000A168C805C00D80229200121A9146AA4240
:101AE00000D9A94620182430391C4A46FEF780FE4A
:101AF000A37940210B43A3714F44A268131C4B44AC
:101B0000A36031680B1C4B4433604A46AD1A002D6C
:101B100000D036E7A368E1688B4200D9E360A27980
:101B200020231343A3710023181C3CBC9046994604
:101B3000A246AB46F8BDC04638B5041C8188006893
:101B4000FEF7E4FF002845D1A3799A0642D55A064C
:101B50000FD5211C243123685878A269012303F092
:101B6000EDF8031C0120002B34D1A37940229343CC
:101B7000A3712068E169FEF73DFF00282AD1256A9C
:101B8000EA7A20231343EB72237B2B77A3891B0A6A
:101B90006B77A37BAB77E37BEB77237CAB76238AF6
:101BA0001B0AEB76A37C2B75638A1B0A6B7501F00D
:101BB00015FEA875030AEB75030C2B76000E6876EC
:101BC000A37920229343A371012322681371206813
:101BD000FFF776F938BDC04610B5041CFFF7ACFF1F
:101BE000002801D10023236010BDC046F0B5574640
:101BF0004E464546E0B4041C0D1C81880068FEF783
:101C000085FF061C002E00D0CBE0A3795AB202203B
:101C1000002A00DAC5E0E268AA4202D2990700D49D
:101C2000151CA26890460023A360002D7DD0236878
:101C300099469F787F02002A14D0681E391C06F04E
:101C40002AF8824601235B4298444046391C06F03C
:101C500022F8824506D37B4241460B40A360ED1A31
:101C600061691AE02169002916D14846FFF7EAFAAE
:101C7000011E012906D1A27980235B421343A3717F
:101C800002208EE0421C06D1A27980235B421343DE
:101C9000A371012085E02061616100292BD100251D
:101CA00046E0A2794346134205D02068FFF7CAFAFE
:101CB000011E04D124E02068FFF782F9011C4A1CB0
:101CC00006D1A27980235B421343A371012068E00F
:101CD000012903D92268D2698A4206D8A2798023D1
:101CE0005B421343A37102205BE06161A368DA19D0
:101CF000A260ED1B01E002229046BD42D1D800E077
:101D00003D1CA3685A19A260EA0510D02068FFF7AD
:101D10004BF9002806D1A27980235B421343A371BB
:101D200002203EE06D0A2D1802E0002500E00025AB
:101D3000A168CB052BD0A269AA4228D0A379590665
:101D400013D5211C243123685878012302F0F6FFB3
:101D5000002806D0A27980235B421343A37101209F
:101D60001FE0A37940229343A371211C24312268F0
:101D700050782A1C012302F09BFF002806D0A2798C
:101D800080235B421343A37101200AE0A561A3688D
:101D9000E1688B4204D9E360A27920231343A37145
:101DA000301C1CBC90469946A246F0BDF0B5574683
:101DB0004E464546E0B482B082469146051C00245A
:101DC0000139884601AE0FE04846311C01226B46BE
:101DD000FFF7CCFC009B012B0AD133786F1C2B70D2
:101DE00001340A2B03D03D1CA045EDDC00E03D1C76
:101DF00000232B70631E9C4160425346184002B082
:101E00001CBC90469946A246F0BDC04600B583B0C2
:101E10006B461870081C6946012201ABFFF78CFD68
:101E200001980138431E984140420123184303B0F2
:101E300000BDC04670B5041C0E1C002506E0311C18
:101E4000FFF7E4FF431C05D001340135207800285A
:101E5000F5D1281C70BDC0460EB4F0B55F4656469D
:101E60004D464446F0B488B0834611AB02CB07938D
:101E70000022904600270E1C3FE1741C3078002899
:101E800000D13EE125280AD05946FFF7BFFF804622
:101E9000031C013301D001218846261C2CE1B31C10
:101EA00072789146302A05D1F31CB678B1460121EB
:101EB000019109E00022019249462D2904D1F31C29
:101EC000B678B146022201921E1C00254B4607E05F
:101ED000AA0055196D00EB181D1C303D33780136F2
:101EE0001A1C303A092AF3D999466C2B01D04C2B95
:101EF00006D10423019919430191327891460136A4
:101F00004B46002B00D1FCE04A46613A192A01D821
:101F1000203BDBB21A1C423AD1B2162952D88A00B1
:101F20007F498A589746079B1A1D07921A68002412
:101F300000E00134135D002BFBD19146019B9B0710
:101F400009D50021884615E020205946FFF75EFF9D
:101F500036182C1C04E00022B246161CB8462F1C72
:101F6000651CBC42F0D35346AA463D1C4746B046CA
:101F70001E1C544648465946FFF75CFF8044B14654
:101F80004646B8462F1C05E020205946FFF73EFF85
:101F900036182C1C651CBC42F6D34746B0464E464C
:101FA000431C00D0A8E08046A6E0079B1A1D0792BC
:101FB00018785946FFF72AFF80469DE00A240AE078
:101FC000102408E048465946FFF720FF804693E07A
:101FD000022400E008240421019A114204D0079A47
:101FE000111D079117680AE0442B04D1079A111DAF
:101FF0000791176803E0079A111D07911768442B92
:1020000006D1002F04DA7F42082301991943019178
:102010000022A846151CB246261C00E01D1C381CD8
:10202000311C05F038FECCB2381C311C05F033FEF3
:10203000071C092C06D907234946782900D12723F4
:102040001C19E4B26B1C303403AA5455002F01D084
:102050000F2BE3D91C1C45465646019A120703D59F
:102060002D2203AB1A550134202398460199C90744
:1020700001D5302290460027022301991940231CE4
:10208000B1462E1C0D1CA24605E040465946FFF7FE
:10209000BDFE3F18231C002D0AD15C1CB342F4D3B3
:1020A000351CA04654464E46C146A8465D4604E04F
:1020B0005446B0465D464E469946013C03AB185D1A
:1020C000291CFFF7A3FE3F18002CF6D1AB4645466E
:1020D0004B46B0465E4605E02020311CFFF796FED9
:1020E0003F18231C5C1CAB42F6D3B34646468046E1
:1020F000021C013200D0B84647444346013300D0A9
:10210000BBE64146013100D14746381C08B03CBC13
:1021100090469946A246AB46F0BC08BC03B01847AF
:10212000B87D00007047C046012817D0002802D0B3
:10213000022824D033E0012A08D1A023DB051A6A43
:1021400001208840011C1143196228E0A023DB050F
:102150001A6A0120884082431A6220E0012A07D1CE
:102160000F4B1A6A01208840011C1143196216E0C6
:102170000B4B1A6A0120884082431A620FE0012A41
:1021800007D1084B1A6A01208840011C11431962CB
:1021900005E0044B1A6A0120884082431A627047A6
:1021A0000000015000000250012814D0002802D085
:1021B00002281ED02AE0002A06D001238B40191CD9
:1021C000A023DB05D96021E001238B40191CA0234B
:1021D000DB0519611AE0002A05D001238B40191C88
:1021E0000B4BD96012E001238B40191C084B19617D
:1021F0000CE0002A05D001238B40191C054BD96047
:1022000004E001238B40191C024B19617047C04642
:102210000000015000000250012808D0002802D020
:10222000022807D008E0A023DB055A6804E0064B2B
:102230005A6801E0054B5A6801238B40101C184076
:10224000431E98417047C0460000015000000250F4
:1022500030B5031C0022134C002002E0910008510D
:102260000132132AFADD00210E4C002502E0013371
:10227000081C011C1A78202AF9D0002A10D0481C0A
:1022800089000B5100E001331A78002A01D02C2A72
:10229000F9D1002A05D01D7001331428E9D100E0DE
:1022A000081C30BD4806001038B50D1C8400134BC7
:1022B000E1580C780020002C1FD0012A0ED002DC3F
:1022C000002A05D018E0022A0BD0032A0FD013E011
:1022D000081C04F06BFD286001200EE02C7001202A
:1022E0000BE0081C04F028FD2860012005E0281CF4
:1022F00005F046F9012000E0012038BD4806001035
:1023000010B5011C0931094C201C05F039F9201CBD
:1023100004F0B6FCC0B2032803D903380022034BF3
:102320001A540122024B1A7010BDC046A0050010BD
:10233000AC04001010B52A4C0020211C0222FFF72B
:10234000B3FF211D01200222FFF7AEFF211C08313F
:1023500002200122FFF7A8FF211C0C3103200222DA
:10236000FFF7A2FF211C103104200122FFF79CFF80
:10237000211C143105200022FFF796FF211C183183
:1023800006200022FFF790FF211C1C3107200222AB
:10239000FFF78AFF211C203108200222FFF784FF6B
:1023A000211C243109200122FFF77EFF211C283146
:1023B0000A200222FFF778FF211C2C310B2001227A
:1023C000FFF772FF211C30310C200022FFF76CFF59
:1023D000211C34310D200322FFF766FF10BDC046DB
:1023E0000C060010024B187941384342584170479F
:1023F00098080010F0B5474680B4424C0020211CDC
:102400000022FFF751FF211D01200122FFF74CFFA1
:10241000211C083102200222FFF746FF211C0C314B
:1024200003200122FFF740FF211C1031042002226B
:10243000FFF73AFF211C143105200122FFF734FF7A
:10244000211C183106200222FFF72EFF211C1C310F
:1024500007200222FFF728FF211C2031082000223C
:10246000FFF722FF211C243109200222FFF71CFF65
:10247000211C28310A200122FFF716FF224D236874
:102480002B60226A2A622148214904F037FF276A1B
:10249000381C204905F0FFFBC6B21F4B1E701F4BB6
:1024A00098465E43F619301C642105F0F4FBC0B277
:1024B0001B4B187064277F4278438619FA23DB0090
:1024C000F618184B1E802668301C124905F0E3FBF5
:1024D000C0B2154B1870434658438619301C64210E
:1024E00005F0D9FBC0B2114B18704743BE19104B11
:1024F0001E70281C211C2C2204F0A5FF04BC904651
:10250000F0BDC04698080010DC0500103D750000C5
:10251000587E00001027000022000010F0D8FFFFB6
:1025200008000010200000101C000010D004001053
:10253000C8040010014B18607047C0460806001020
:10254000F8B5041C2C233C4AD35C012B01D900F0C4
:10255000BFFF2378242B04D03848394904F0CEFE3D
:1025600068E0201C04F08CFB061C0023002009E01E
:10257000711E61180A780A2A01D00D2A01D108704B
:10258000013E0133012BF3DDB01E201804F0A2FC44
:10259000021C033E0023012102E0655C6B40013117
:1025A000B142FADB834203D02448264904F0A6FE58
:1025B000601C254904F052FB002803D1201CFFF7C2
:1025C0009FFE37E00023A371A6193370E01DFFF7CB
:1025D0003FFE051C0334201C1C4904F03FFB00286F
:1025E00006D11B4B1B68DA0702D5281CFFF7A2FE99
:1025F000201C184904F032FB00281BD1144B1B6827
:10260000DA0617D5144B1B78022B10D108E0A30073
:10261000D85904F0EDFB301C04F0EAFB013402E071
:1026200000240E4F0E4EAC42F1DB04F073FC281C6C
:10263000FFF7E0FEF8BDC046E80B00103D75000056
:10264000687E0000847E0000C07E0000C87E00001E
:1026500008060010CC7E0000A404001048060010FC
:10266000D07E000008B5034B996A012004F0E8F918
:1026700008BDC046E80B001038B52DE0012004F07D
:10268000B1FA051C041E27D024280AD10022154BBC
:102690001A60154B1B78012B03D11448144904F020
:1026A0002DFE104A1368134AD554FF22520093425C
:1026B00002DC01330B4A13600B4A1378012B02D161
:1026C000281C00F0BDFC0D2C06D1064B1B680948E8
:1026D0000022C254FFF734FF012004F07DFA0028E5
:1026E000CCD138BDA8040010A40400103D75000032
:1026F0000C8700009806001038B5174B1B78002B8C
:1027000028D1164B1B78022B07D01548154904F029
:1027100037FF0122104B1A701CE00422124B1A7072
:102720002423124AD05C12490D2204F039FA0E4CCF
:10273000094D01E0FFF7A0FF2378002B02D02B7892
:10274000002BF7D0044B1B78002B03D10448094918
:1027500004F016FF024838BDAC040010040000105D
:10276000A0050010D47E0000E8040010E80B001063
:10277000DC7E0000EC7E000008B58020FE2100F029
:10278000B7F90020142103F0D3FD08BD10B584B0C3
:10279000194B1B78012B2AD90023002103E001AA41
:1027A000D1540133DBB2082BF9D98020F52100F098
:1027B0009FF90020142103F0BBFD01AC8020211CF7
:1027C000032200F0B5F920780002637818430B4B20
:1027D00018400B4B584300140A4BC0180A4B984240
:1027E00000DD181CC343DB17184080B200E0002056
:1027F00000B204B010BDC04604000010FCFF000091
:10280000D4300000A8FDFFFF102700008023DB0567
:102810005B68FF221340083B502B00D9B8E09B00B7
:102820005E4AD3589F465E4B00221A601A68511CBC
:1028300019605C4B9A5CD2B28023DB059A60282237
:102840009A610122584B1A60A6E00022574B1A6089
:10285000534A1368591C1160524AD25CD2B2802389
:10286000DB059A6028229A6102224F4B1A6093E09E
:102870004D4B1B68012B0CD1494A1368591C116040
:10288000484AD25CD2B28023DB059A600422464BD0
:102890001A6008228023DB059A617DE0404B1A68AC
:1028A000434B1B689A420DD23D4A1368591C116074
:1028B0003C4AD25CD2B28023DB059A6004223A4BB8
:1028C0001A6012E03B4B1B68002B07D020228023AC
:1028D000DB051A600322344B1A6006E00522324BF6
:1028E0001A6010228023DB051A6008228023DB0592
:1028F0009A6151E02F4B1B68012B04D104228023E5
:10290000DB059A6103E004228023DB051A600822BC
:102910008023DB059A613FE0244B1A68511C196043
:102920008021C9058868C0B2234988541A68214BA0
:102930001B689A4206D204231B4A13608022D205E8
:10294000136006E00522184B1A6004228023DB0581
:102950009A6108228023DB059A611DE0134B1A68F7
:10296000511C19608023DB059868C0B21249885455
:1029700005210D4A116010221A6008229A610BE0AD
:1029800008228023DB059A610522074B1A6003E0C9
:1029900008228023DB059A617047C046F87E00005C
:1029A000BC040010EC080010B4040010B0040010C7
:1029B0000C090010C4080010C808001010B520222F
:1029C0008023DB051A6000220A4B1A6000230949A4
:1029D00009480A4C05E00268012A07D0A34207D83B
:1029E00001330A68012AF6D9002002E0012000E044
:1029F000002010BDD80B0010B4040010FEFFFF0033
:102A00008023DB0510221A6008229A61191C10220B
:102A10000B681A42FCD101207047C04670B51C4BB0
:102A20005A6802210A435A6080229D5820242C4370
:102A30009C50184B90229C583F25AC439C509C586E
:102A40000C439C509E588024E40026439E509422C0
:102A50009E58AE439E509D582943995099580C4317
:102A60009C508023DB056C229A6132225A611A61E4
:102A7000022803D1A0228023DB05DA6080225201E4
:102A8000054B1A6040228023DB051A60012070BDCF
:102A9000008004400040044000E100E010B5002345
:102AA0000F4A13600F4A13600F4A1360FFF786FF47
:102AB000041E012C03D0FFF7A3FF00240EE0002228
:102AC0000A4B1A601A1C064905E00B68052B02D157
:102AD000FFF796FF02E01368092BF6D9201C10BD02
:102AE000B4040010B0040010BC040010D80B001097
:102AF00008B50A4B18705970094B1B78DA0704D5D2
:102B000008480649022204F04BFA0222064B1A60DA
:102B10000022064B1A60FFF7C1FF08BDEC08001049
:102B2000B8040010448000000C090010C408001014
:102B300038B50D1C141C012318430E4B18700E4B96
:102B40001A600E4B01221A60FFF7A8FF00230C4AFF
:102B500003E0D05CE8540133DBB2A342F9D3094A65
:102B60001278910704D5084805491A1C04F018FA90
:102B700038BDC046EC080010C40800100C09001055
:102B8000C8080010B80400104C80000008B5124BB3
:102B9000802298588021C90101439950985880217A
:102BA000C9000143995098584021014399509858C1
:102BB000802149020143995001229A6772B6392255
:102BC000064B1A60064B1B6883F30888054B1B688D
:102BD00002480549984708BD0080044010090010CC
:102BE0000000FF1F0000001024090010BFF34F8FEA
:102BF000024A034BDA60BFF34F8FFEE70400FA0589
:102C000000ED00E0F0B55F4656464D464446F0B450
:102C100085B00023002203E06946CA540133DBB2C9
:102C20000F2BF9D900229246304B9946304DA846D9
:102C300029E0072751467D1AEDB253460833DBB22F
:102C40009C46012200234C0017E0215A0A4210D072
:102C50001E1C4F46FF5C291C002F00D061464746D2
:102C6000BE5D0127B7403E1C6F467F5C3E436F460A
:102C70007E54520092B20133DBB20F2BE5D9564697
:102C80000136F6B2B24651460729D2D9194B702205
:102C90001A70C8225A7080229A70174B1B78002B2A
:102CA00003D0F122134BDA7002E0F022114BDA70FC
:102CB0006022104B1A71002305220E4C06E0511CB5
:102CC0006D46E85CA0540133DBB2CAB20F2BF6D9D3
:102CD0000A4B1A6000220A4B1A60FFF7DFFE05B0AC
:102CE0003CBC90469946A246AB46F0BD84810000AC
:102CF00074810000EC080010490900100C09001054
:102D0000C4080010F0B54F464646C0B485B01A4B13
:102D10001A780023002A1BD0013A174B1A7026E0BC
:102D20001A1C6046C156002902DA4D461349CD549B
:102D3000B95C4900895B50006D464153A05C002896
:102D400003D052004046014351530133DBB209E046
:102D50000A48844600218946071C094E094C8022F6
:102D6000D2019046072BDBD96846FFF74BFF05B031
:102D70000CBC90469946F0BD4A0900103409001079
:102D8000748000004C09001010B500220F4B1A701F
:102D900000230F4902E0CA540133DBB2072BFAD9F2
:102DA0000C4B70221A70C8225A7080229A70F0223E
:102DB000DA7060221A710522074B1A600024074B53
:102DC0001C60FFF76BFE064B1C7010BD490900101C
:102DD00034090010EC0800100C090010C4080010A1
:102DE0004A090010F8B50023114D20241149002292
:102DF00003E0EC54CA540133DBB2072BF9D90022AB
:102E000000210B4D0B4E012709E02E2B02D1531E42
:102E1000F75402E0541CAB54E2B20131C9B2072AA4
:102E200002D8435C002BF0D1FFF76CFFF8BDC04621
:102E3000340900104C09001008B5FFF7D3FF102229
:102E4000014B1A7008BDC0464A090010F0B547464C
:102E500080B484B0052800D9C2E08000624B1B58C2
:102E60009F465A00684611520133DBB202E000234C
:102E700001214942072BF4D96846FFF7C3FE002021
:102E80005A4903F055FAABE05A00694654520133EF
:102E9000DBB202E0331C4446AC40072BF4D9684651
:102EA000FFF7B0FE301C391C03F042FA0135EDB2D9
:102EB00005E00025002601229046FA277F000F2D0D
:102EC000E8D98DE05A00684611520133DBB201E0C7
:102ED00000230021072BF5D9002188460026012771
:102EE00018E03B1CA34068462A5A13432B52FFF7B5
:102EF00089FE301CFA21490003F01AFA0134E4B2C9
:102F000002E0341C424655000F2CEAD943460133F7
:102F1000DBB298464346072BF3D90020FA21C900BB
:102F200003F006FA5CE05A00684611520133DBB246
:102F300001E000230021072BF5D900218846002657
:102F4000012717E03B1CA34068462A5A13432B5223
:102F5000FFF758FE301C142103F0EAF90134E4B203
:102F600002E0341C424655000F2CEBD94346013396
:102F7000DBB298464346072BF3D90020FA2189009B
:102F800003F0D6F92CE05A00684611520133DBB247
:102F900001E000230021072BF5D90020002501279F
:102FA0001AE03B1CA340694673526846FFF72AFEAD
:102FB000281C03F017FE0134E4B202E02C1C424648
:102FC00056000F2CEDD943460133DBB2984600E0A2
:102FD000A8464346072BF1D9512801D07128F7D1D3
:102FE00004B004BC9046F0BD5C8000008813000073
:102FF00008B5002003210122FFF796F800200421E4
:103000000122FFF791F8002005210122FFF78CF83B
:10301000002003210122FFF7C7F80020042101222C
:10302000FFF7C2F8002005210122FFF7BDF808BD17
:1030300008B5031C0A1C0020191CFFF7B5F808BDD1
:10304000044920224B691A42FCD0024B1860002030
:103050007047C0460080004010B50A4B1B680A4A02
:103060001268934205DA094A12685C1C05490C6033
:10307000D054064B1A68034B1B68D31800221A70F1
:1030800010BDC046D40400104C0E0010E004001027
:103090000CB410B582B004AA08CA0024074B1C6007
:1030A000074B1960074B186001920748049904F018
:1030B00065F802B010BC08BC02B01847D404001078
:1030C0004C0E0010E004001059300000F0B54746E7
:1030D00080B486B0041C0E1C151C1F1C00281ADAB4
:1030E0004442A04603AC2D23237000236370201CB0
:1030F00004F038FA4046291C04F0CAFD061C40467C
:10310000291C04F0C5FD0091381C0621221C331C2B
:10311000FFF7BEFF0EE0111C04F0BAFD8046201C34
:10312000291C04F0B5FD0091381C0621321C4346D1
:10313000FFF7AEFF06B004BC9046F0BD08B501F045
:10314000EFFC01F0E3FC00280CD00022064B1A70C3
:1031500000200649FEF73EFA002803D0044805493E
:1031600004F0CCF808BDC046680900107C090010C6
:1031700041300000C4810000F0B5474680B4184CCF
:10318000A54401F0C3FC002823D01648FFF72AFE0F
:1031900001A815490122FEF733FA002819D1134E70
:1031A000134B9846134F301C282101AAFEF7FEFD51
:1031B000041E09D00D4D4046391C2A1C04F09EF80F
:1031C000281C282101F0ACFE002CECD101A8FEF750
:1031D00003FD8A239B009D4404BC9046F0BDC0467D
:1031E000D8FDFFFFDC810000E8810000B00B00107B
:1031F00041300000F881000010B582B00C4C0D4B3E
:103200001A880D4B1B780D4909780091201C0C4938
:10321000FEF722FE0B4B1A780B4B1B780B490978F3
:103220000091201C0A49FEF717FE02B010BDC046EF
:10323000981100102000001008000010220000105B
:10324000008200001C000010D0040010C804001010
:103250001882000010B501F059FC002834D01B483A
:103260001B491222FEF7CCF9021E04D019481A4954
:1032700004F044F828E0154C201CE168FEF7B6FC89
:10328000201C1649FEF7E8FD201C1549FEF7E4FD59
:10329000201C1449FEF7E0FD201C1349FEF7DCFD5D
:1032A000201C1249FEF7D8FD114B1A783032201C31
:1032B0001049FEF7D1FDFFF79FFF201C0E49FEF7D6
:1032C000CBFD201CFEF738FC10BDC0469811001045
:1032D0002882000041300000348200005C8200003F
:1032E00098820000B0820000D0820000E0820000DE
:1032F00004000010FC82000010830000F0B585B0CF
:10330000114B1B78002B1CD101F000FC002818D0B9
:103310000E4F0F4E0F4D3388684610213A1CFFF7B1
:10332000B7FE281C69460122FEF76AF9041E06D181
:103330000848FEF751FC064B1A8801321A80002C0F
:10334000E9D005B0F0BDC046D204001020830000D3
:1033500006000010700F001010B588B0324B1B78BB
:10336000002B5FD101F0D2FB00285BD000222F4B55
:103370001A702F4B1B8804A810212E4AFFF788FED5
:103380002C232D4AD35C012B06D9294B1B88684678
:1033900010212A4AFFF77CFE254B1A8801321A8039
:1033A000274804A90A22FEF72BF9021E04D025485B
:1033B000254903F0A3FF18E001221B4B1A701422C9
:1033C000224B1A70FFF718FF214C201C21496A4636
:1033D0001232FEF741FD201CFEF7AEFB002204ABCB
:1033E0005A7268461230FFF727FD2C23124AD35C2D
:1033F000012B17D9184869460A22FEF701F9021E67
:1034000004D01048104903F079FF0BE0FFF7F4FEF9
:103410000F4C201C11496A460232FEF71DFD201C8C
:10342000FEF78AFB08B010BDD20400106809001036
:103430000600001030830000E80B001040830000FD
:10344000700F00104130000050830000D9040010BC
:103450009811001078830000280C00109C83000055
:1034600010B5144B1B78002B22D00022114B1A7080
:103470001148FEF7B1FB2C23104AD35C012B02D973
:103480000F48FEF7A9FBFFF7B7FE0E480E49FEF7FF
:10349000E3FC2C23094AD35C012B01D9FFF7ACFED6
:1034A000084C201C0949FEF7D7FC201CFEF744FB02
:1034B00010BDC046D2040010700F0010E80B0010C1
:1034C000280C001098110010C0830000D883000061
:1034D00008B5021C064B1B78002B08D02C2305498D
:1034E000CB5C012B03D904480449FEF7B5FC08BDA9
:1034F000D2040010E80B0010280C001024860000F5
:1035000010B582B01B4C201C1B4903F0F7FE201C99
:103510001A4903F0F3FE201C194903F0EFFE201CAA
:10352000184903F0EBFE184B1A783032201C17496B
:1035300003F0E4FE164B1A88164B1B7816490978DF
:103540000091201C154903F0D9FE154B1A78154B34
:103550001B78154909780091201C144903F0CEFE10
:10356000FFF7CAF8021C201C114903F0C7FE02B085
:1035700010BDC0464130000098820000A4850000C4
:10358000D0820000E082000004000010FC820000F5
:10359000200000100800001022000010008200002F
:1035A0001C000010D0040010C8040010C0850000EA
:1035B000D4850000F0B5474680B482B08046002430
:1035C000094F0A4E0A4D09E06300DB5B4246009258
:1035D000301C291C221C03F091FE0134072CF3DD62
:1035E00002B004BC9046F0BD00160010413000004F
:1035F000F485000038B5084D084B1A68084C281CA3
:103600000849231C03F07AFE074B1A68281C074957
:10361000231C03F073FE38BD413000001816001063
:103620000C87000000860000141600100C860000B5
:1036300008B5031C034A12680348044903F05EFE00
:1036400008BDC046600F0010413000002086000019
:1036500038B5051C0F4C2068642104F019FB021CCE
:103660000D480E4903F04AFE2068642104F010FB67
:103670000C1E092C02DC3020FFF7E2FC002C02D1EA
:103680003020FFF7DDFC04480549221C2B1C03F009
:1036900035FE38BDC41300104130000028860000FC
:1036A0003086000038B5051C074B1868074C0849E0
:1036B0006422231CFFF70AFD06480749221C2B1C25
:1036C00003F01CFE38BDC046941100105C090010C8
:1036D00038860000413000004086000038B5051CE7
:1036E000074B1868074C08490A22231CFFF7EEFC19
:1036F00006480749221C2B1C03F000FE38BDC046BB
:10370000500F0010680F00104C8600004130000080
:103710005486000038B5051C104C0023E05E64217F
:1037200004F0B6FA02B20E480E4903F0E7FD00239A
:10373000E05E642104F0ACFA0CB2092C02DC30200B
:10374000FFF77EFC002C02D13020FFF779FC044803
:103750000549221C2B1C03F0D1FD38BD580900106F
:1037600041300000608600003086000008B5154B2F
:103770001A6801321A60144B1A6801321A60134A2F
:1037800013780133DBB21370632B0DD900220F4B7A
:103790001A700F4B1A6801321A600E4B1B78002BFF
:1037A00002D0013B0B4A13700B4B1B78022B07D145
:1037B00000201D21FEF730FD011C0420FFF738FC1E
:1037C00008BDC046C0040010D80B0010DD0B00106F
:1037D00020160010E80400100400001070B50D4B16
:1037E0001D880D4B18780D4B1C780D4B19780D4B1F
:1037F0001A780D4B1B780D4EAD196D064005284308
:1038000024042043C9020843520110435B081843B3
:1038100070BDC046200000100800001022000010FB
:103820001C000010D0040010C804001044F8FFFF72
:10383000084B1B78002B0BD1074B084A1968116005
:103840000749084A11600121024A117000221A60DA
:103850007047C046D1040010600F00106C090010C2
:10386000F1D8FFFFC013001000B583B0FFF774FD5F
:10387000284B1B78002B4AD02023274AD35C002BEF
:1038800002D0012B04D006E06622244B1A7002E01D
:103890006D22224B1A7021231F4AD35C002B02D0C9
:1038A000012B04D006E046221D4B1A7002E0432291
:1038B0001B4B1A701A4B1B78184A12780092194841
:1038C00019491A1CFEF7C8FA2C23134AD35C002BA3
:1038D0000BD02023D35C9A00D318144AD2180F4B74
:1038E0001B7810481249FEF7B7FA124B1B78012BD0
:1038F00003D90C481049FEF7AFFA0A480F49FEF702
:10390000ABFA054B1B7A032B01D1FFF791FF03B0F4
:1039100000BDC046D2040010E80B00107009001072
:10392000DC0B0010700F0010688600000C00001007
:10393000AC86000004000010F4860000F085000052
:103940000023044A13600449044A1160044A1370B6
:103950007047C0466C090010F1D8FFFFC01300107B
:10396000D1040010F0B55F4656464D464446F0B4CB
:10397000B3B0FFF7E5FFE14A8023D158E0480143A7
:10398000D150FEF7CFFB00200021FEF745FC0028B8
:1039900002D10222DB4B1A70FFF72AFB02F0E6FB92
:1039A000FCF7CCFDD84B0322B4215A50B8215A5011
:1039B0000221BC229950D54B1868642104F06BF9A0
:1039C000D34B984210D80202120A013AD14B5A60E6
:1039D000D14A106A0002000AC0210906014311629F
:1039E00000229A6007221A60FCF7FEFECB4B587843
:1039F000596803F025F8C54B1868642104F04BF9A9
:103A0000421E0020012102F057FE002002F08EFD30
:103A1000C34C201CC34903F071FC0120FEF7FEFFDC
:103A2000201CC14903F06AFCFFF7AEF90420FFF740
:103A30000DFABE48FFF7D6F90020BD4902F078FC28
:103A4000BC48FFF7CFF90020FA21890002F070FC92
:103A5000B948FFF7C7F9B948FCF70CFD002300226D
:103A600004E09900B6480A500133DBB2022BF8D9C2
:103A7000B448FFF7B7F9FCF743FCFCF74FFCC8204C
:103A8000400002F0F1FBCC20FCF76AFC3C2002F085
:103A9000EBFB4420FCF764FC3C2002F0E5FB994B77
:103AA0001B78022B01D1FEF767FEA748FFF79AF9B2
:103AB000944B1B78012B02D90122A44B1A70A34B03
:103AC0001B78012B02D102F00DF901E001F0DCFFBF
:103AD0009F48FFF76FFD00239E4A13609E4A1370B4
:103AE0000A219E4A11709E4A13609E4A9E4B1A609C
:103AF0009E48FFF777F9FFF721FB9D48FFF772F922
:103B0000FFF73AFB854B5B7A012B02D0022B05D0E5
:103B100007E0824BDA68974B1A6002E00122954B6E
:103B20001A607E4B1B7D012B02D0022B05D007E0D3
:103B30007A4B9A69904B1A6002E001228E4B1A6010
:103B4000764B1B7A022B02D101228C4B1A608C48D7
:103B5000FFF748F9FEF786FD2D23704AD05CFEF78B
:103B6000E9FC884B00229A604E2119731A61572193
:103B700019759A61DA61844B1A620020834902F058
:103B8000D7FBFEF779FD8248FFF72CF9FFF762FBC0
:103B9000FFF7B4FB5B4B1B78022B02D1012003F033
:103BA00067FA0120FCF7C4FD012801D101F074F986
:103BB000FEF7A2FD021C774C201C7749FEF74CF95A
:103BC000201CFDF7B9FF7548FFF70CF90021884666
:103BD00000221F9200231E930020229020915D4A14
:103BE000914693466E488246FEF746FD49460B686D
:103BF000042B01D800F00FFD00235A461360534BED
:103C00001B78012B02D102F083F801E001F04EFF96
:103C100001F076FF01F094FF624B186021233F4AC8
:103C2000D35C002B09D1C3001818052104F030F82B
:103C3000C8231B01C0185B4B186001F09DFF5A4B55
:103C40001860474B196840181860444A1378013BC4
:103C5000DBB21370002B00D0E6E00A223F4B1A7053
:103C60000A2104F015F8514B186001F0F7FF504B92
:103C700018602023294AD35C012B06D152465043B9
:103C80004C4904F005F84A4B1860494A4A4B1B68F6
:103C90001068C31A13600021314A1160324A126859
:103CA000934201DD304A13600620FCF71DFC80B210
:103CB000424B1880424B58438012424B5843FA21E2
:103CC000890003F0E5FF404B186000243F4E3C4F55
:103CD0001B4D0AE0305DFCF707FC0004000C784344
:103CE0008012A30058510134E4B2022CF2D9209979
:103CF00000296DD0012974D082E0C04600800440C4
:103D00001F0001E00400001000400440880400107F
:103D1000FFFFFF0010E000E000ED00E0E80B001006
:103D20004130000004870000108700001C8700005D
:103D3000DC0500002887000034870000405489001B
:103D4000540F0010408700004C870000D80400107A
:103D50000C870000C0040010DD0B0010E40B001005
:103D600074090010F1D8FFFFC0130010588700003D
:103D700060870000DC040010E4040010CC04001094
:103D80006C870000DC0500100C060010980800008D
:103D9000788700009811001084870000A487000035
:103DA000102700009411001064090010C4130010C3
:103DB000600F0010288000006C090010DE0B00105E
:103DC000E40C0000D6100000BC1300101800001016
:103DD00003200121FFF72CF905200021FFF728F926
:103DE0000EE0DB4B1B78002B03D003200021FFF7F4
:103DF0001FF905200121FFF71BF901235B422093E6
:103E0000D44B1B78012B0CD1FEF7ECFA002804D020
:103E100004200021FFF70CF903E004200121FFF743
:103E200007F9209A0132209243460B2B00D90DE16D
:103E30009B00C94AD3589F46C84B1B682FA80C212A
:103E4000C74AFFF725F92FA8FEF7CCFFFEE0C54BC8
:103E50001B682FA80C21C44AFFF71AF92FA8FEF7F8
:103E6000C1FFF3E0C14B18680A2103F011FFC04EF7
:103E7000C04C311C0A22231CFFF728F9BE4B1868DE
:103E8000BE4D311C0A222B1CFFF720F900952FA8EC
:103E90000C21BB4A231CFFF7FBF82FA8FEF7A2FF5B
:103EA000D4E0B84B1C68201C642103F0F1FE051C13
:103EB000201C642103F0ECFE00912FA80C21B24AD3
:103EC0002B1CFFF7E5F82FA8FEF78CFFBEE0AF4BE9
:103ED0001F68381CE121090103F0DDFEFF26341CB8
:103EE0000440AB4D6543ED19281C3C2103F0D3FE83
:103EF00006403301F31A9B005D19009601952FA827
:103F00000C21A44A231CFFF7C3F82FA8FEF76AFF71
:103F10009CE0A14B1C68201CFA21890003F0B8FE2C
:103F2000051C201CFA21890003F0B2FE00912FA885
:103F30000C219A4A2B1CFFF7ABF82FA8FEF752FF73
:103F400084E0279804B2201C642103F0A1FE05B28E
:103F5000201C642103F09CFE09B200912FA80C21C3
:103F60008F4A2B1CFFF794F82FA8FEF73BFF6DE05C
:103F70008C4DAC68201C514603F08AFE4E1D2D7BF3
:103F8000201C514603F084FE041C301C0A2103F05F
:103F90007FFE009001952FA80C21834A231CFFF778
:103FA00077F82FA8FEF71EFF50E07E4D2C69201CED
:103FB000514603F06DFE0E1C32362D7D201C5146FD
:103FC00003F066FE041C301C642103F061FE0090C7
:103FD00001952FA80C21754A231CFFF759F82FA82B
:103FE000FEF700FF32E02398514603F051FE041C17
:103FF0002398514603F04CFE00912FA80C216C4AE7
:10400000231CFFF745F82FA8FEF7ECFE1EE0654BDA
:10401000DC69201C514603F03BFE051C201C514668
:1040200003F036FE00912FA80C21624A2B1CFFF7EB
:104030002FF82FA8FEF7D6FE08E02FA80C215E4A25
:10404000249BFFF725F82FA8FEF7CCFE01F06AFCB1
:104050000020FCF76DFB041C0120FCF769FB051C2C
:10406000031C1E998C4223D01E94002C20D1424662
:104070000132D2B29046374A1278012A05D8424618
:10408000062A02D10132D2B2904600220B214046CC
:10409000814252415242104080462C2247498A5C5C
:1040A0001E94002A04D1062802D91E9400218846B5
:1040B0001F9A93420DD01F95002B0AD1244B1B78D9
:1040C000002B03D0FFF7CCF91F9502E0FFF7CCFBE4
:1040D0001F952E4B1B682298984200D19BE2374BCC
:1040E0001B7A022B0AD1364A1368013B1360002B5E
:1040F00004D10022314B1A72FFF79AFB2F4B5B7AE7
:10410000012B02D0022B10D01BE02E4A1368013B7A
:104110001360002B15D10022284B5A720C4B1B78D0
:10412000002B0ED1FFF7A0FB0BE0094B1B78002BF7
:1041300007D10A4B1A68214B1B699A4201D3FFF73A
:1041400093FB1E4B1B7D012B3ED0022B4CD057E026
:10415000D20400100400001094810000600F0010D1
:10416000AC870000C0130010B48700009411001049
:104170004C8600005C090010500F0010680F001002
:10418000BC870000C4130010C48700002016001074
:10419000F0F1FFFFD0870000BC130010E0870000A3
:1041A000EC870000DC050010FC8700000888000098
:1041B00014880000208800002C880000E80B001004
:1041C000CC040010DC040010B54A1368013B1360F6
:1041D000002B15D10022B34B1A75B34B1B78002B63
:1041E0000ED0FFF73DF90BE0AF4B1B78002B07D04B
:1041F000AE4B1A68AB4BDB699A4201D2FFF730F93C
:104200003C23A84AD35C012B03D12498FCF7C0F9C6
:1042100003E0A64B1868FCF7BBF90022A44B1A7008
:10422000A44B1B682293FCF779F8C820400002F0E9
:104230001BF8CC20FCF794F83C2002F015F8BE20C7
:10424000FCF78EF83C2002F00FF86C46BA34201CC4
:104250000221FCF7C1F80021635E9A00D3185B00CD
:10426000DA17120FD3181B11934A136021228D49BC
:104270008A5C002A08D1D800C018052103F008FD87
:104280004130FF308C4B1860FCF748F8C8204000E4
:1042900001F0EAFFCC20FCF763F83C2001F0E4FFDA
:1042A0004420FCF75DF83C2001F0DEFF834B1B78D7
:1042B000022B03D1FEF76AFA80B22790804B186870
:1042C00080496422804BFEF701FF7B4B18687F49D1
:1042D0000A227F4BFEF7FAFE2023724AD45C002CA0
:1042E0000BD17C4B186A514603F0D2FC7A4B5843F1
:1042F000514603F0CDFC249005E0764B186A5146F8
:1043000003F0C6FC2490002C0ED1744B9869142144
:1043100003F0BEFC724B5843514603F0B9FC8300D6
:104320001818800023900DE06C4B9869142103F05D
:10433000AFFC6C4B5843514603F0AAFC830018189D
:10434000800023902C23574AD35C002B00D1D5E06A
:10435000584B1B682893644B1B681D93534B1B6879
:104360002993624B1F68624B1E685D689C685B4BBB
:104370001A682A9298682190197B2B911A692592C4
:10438000187D2C90DB692693FEF72CF82D901D9854
:10439000642103F07DFC00901D98642103F078FCFB
:1043A0000191494B02934A4B039329990491381C7C
:1043B000FA21890003F06CFC0590381CFA21890071
:1043C00003F066FC0691301CFA21890003F060FCC2
:1043D0000790301CFA21890003F05AFC0891281C30
:1043E000FA21890003F054FC0990281CFA21890065
:1043F00003F04EFC0A91201CFA21890003F048FCCE
:104400000B90201CFA21890003F042FC0C912A9A9F
:104410000D922198514603F03BFC0E902198514695
:1044200003F036FC0F912B9B10932598514603F017
:104430002FFC11902598514603F02AFC12912C98DC
:1044400013902398514603F023FC1490239851466F
:1044500003F01EFC15912698514603F019FC1690A6
:104460002698514603F014FC1791249918912D9A1F
:104470001992279B1CB2201C642103F009FC00B296
:104480001A90201C642103F003FC09B21B91194807
:1044900080214900184A289BFEF7FAFD90E0C046AB
:1044A000E4040010E80B0010D2040010600F0010AC
:1044B0001C16001020160010500F001004000010F1
:1044C00094110010388600005C0900104C86000032
:1044D000680F00100C06001028800000DC0500109A
:1044E000F42C000058480000C4130010BC13001046
:1044F000540F0010500E001034880000474B1B680A
:104500001D93474B1F68474B1E685D689C68464B70
:104510001B6821931D98642103F0BAFB00901D983D
:10452000642103F0B5FB0191404B0293404B039390
:10453000404B1B680493381CFA21890003F0A8FB48
:104540000590381CFA21890003F0A2FB0691301C6B
:10455000FA21890003F09CFB0790301CFA218900A6
:1045600003F096FB0891281CFA21890003F090FBC8
:104570000990281CFA21890003F08AFB0A91201C6B
:10458000FA21890003F084FB0B90201CFA2189009A
:1045900003F07EFB0C91279804B2201C642103F0E9
:1045A00077FB00B20D90201C642103F071FB09B26F
:1045B0000E91214880214900204A219BFEF768FD89
:1045C0001F4B1B78002B04D01E481F491A4A02F0CB
:1045D00095FE1E4B1B78002B1DD01D4A1388013BF6
:1045E0009BB21380002B16D11A4B5A8C184B1A8091
:1045F000194B1A6801321A60184819490E4AFDF71A
:104600002BFC094B1B683F22191C91438B4202D1A2
:104610001248FDF791FA30BFFFF7E6FAC413001015
:10462000BC130010540F0010201600105C0900107D
:10463000680F0010600F0010500E0010B4880000CA
:10464000D304001041300000F8810000D2040010B3
:104650001E000010E80B0010C4040010700F0010C2
:1046600020840000F8B54F464646C0B40D1C4023D8
:104670009946202398461027461C047863B2002BE5
:1046800005DA002011210122FDF78EFD04E0002053
:1046900011210022FDF788FD00200E210122FDF7E7
:1046A00083FD00200E210022FDF77EFD4B462342B4
:1046B00005D0002011210122FDF776FD04E0002045
:1046C00011210022FDF770FD00200E210122FDF7CF
:1046D0006BFD00200E210022FDF766FD43462342BC
:1046E00005D0002011210122FDF75EFD04E000202D
:1046F00011210022FDF758FD00200E210122FDF7B7
:1047000053FD00200E210022FDF74EFD274205D06B
:10471000002011210122FDF747FD04E000201121B6
:104720000022FDF741FD00200E210122FDF73CFD96
:1047300000200E210022FDF737FD230705D50020BC
:1047400011210122FDF730FD04E00020112100229B
:10475000FDF72AFD00200E210122FDF725FD002096
:104760000E210022FDF720FD630705D50020112151
:104770000122FDF719FD04E0002011210022FDF7C0
:1047800013FD00200E210122FDF70EFD00200E2159
:104790000022FDF709FDA30705D500201121012204
:1047A000FDF702FD04E0002011210022FDF7FCFCD2
:1047B00000200E210122FDF7F7FC00200E2100222F
:1047C000FDF7F2FCE30705D5002011210122FDF7DA
:1047D000EBFC04E0002011210022FDF7E5FC0020A5
:1047E0000E210122FDF7E0FC00200E210022FDF742
:1047F000DBFC013D301C002D00D03DE70CBC904699
:104800009946F8BD70B5051C0C1C00201121012231
:10481000FDF7CAFC00E01D1C00201021FDF7FCFC88
:10482000061C701E864100200E210122FDF7BCFCF3
:1048300000200E210022FDF7B7FC7600F6B2002022
:104840001021FDF7E9FC002801D00136F6B2002066
:104850000E210122FDF7A8FC00200E210022FDF709
:10486000A3FC760000201021FDF7D6FC002801D023
:104870000136F6B200200E210122FDF795FC002042
:104880000E210022FDF790FC7600F6B200201021E8
:10489000FDF7C2FC002801D00136F6B200200E213F
:1048A0000122FDF781FC00200E210022FDF77CFC97
:1048B0007600F6B200201021FDF7AEFC002801D0F2
:1048C0000136F6B200200E210122FDF76DFC00201A
:1048D0000E210022FDF768FC7600F6B200201021C0
:1048E000FDF79AFC002801D00136F6B200200E2117
:1048F0000122FDF759FC00200E210022FDF754FC97
:104900007600F6B200201021FDF786FC002801D0C9
:104910000136F6B200200E210122FDF745FC0020F1
:104920000E210022FDF740FC7600F6B20020102197
:10493000FDF772FC002801D00136F6B200200E21EE
:104940000122FDF731FC00200E210022FDF72CFC96
:104950006B1C2E70013C002C00D05CE770BDC04683
:1049600000B583B000200F210122FDF71DFC684631
:1049700007300121FFF746FF03B000BD30B583B01B
:104980000B4C6D4607350BE0281C0121FFF73AFF61
:104990002B78FF2B06D00020642101F081FC013C24
:1049A000002CF1D1631E9C41E0B203B030BDC04683
:1049B0008813000010B582B000200F210022FDF7FF
:1049C000F3FB684607300121FFF71CFFFFF7D6FF16
:1049D000041E02D1FFF7C4FF00E00124201C02B036
:1049E00010BDC04630B583B0041C0D1C43B2002B73
:1049F00008DA7F231C4037200021FFF7F3FF031C58
:104A0000012B35D8FFF7ACFFFFF7D4FF031CFF20C5
:104A1000002B2DD0402323436A4613702B0E537076
:104A20002B0C93702B0AD37015719523002C00D09A
:104A30000123082C00D187236A465371684606215A
:104A4000FFF710FE0C2C04D1684607300121FFF758
:104A5000D9FE0A246D460735281C0121FFF7D2FE36
:104A6000287843B2002B03DA013CE4B2002CF3D1E6
:104A700003B030BD30B583B0051C0C1CFFF77EFFC2
:104A800000281BD001A804700121FFF7EBFD0120D5
:104A9000FD2C13D0281C80218900FFF7E3FD01AC19
:104AA000201C0221FFF7AEFE201C0121FFF7AAFE09
:104AB00023781F20184005384342584103B030BDC9
:104AC000F0B583B0071C0E1CFA24A40001AD0BE066
:104AD000281C0121FFF796FE2B78FF2B06D1002022
:104AE000642101F0DDFB013C002CF1D101AB1A780F
:104AF0000020FE2A08D1381C311CFFF783FE01A8D4
:104B00000221FFF77FFE012003B0F0BD08B50020B1
:104B10001B21FDF781FB0138431E9841C0B208BD3F
:104B200008B500201B210022FDF7FEFA08BDC04693
:104B300030B583B0124B1D78032400281AD11B21F5
:104B4000FDF76AFB012815D006232C1C9C43EB07BC
:104B500010D43A200021FFF745FF002801D001239F
:104B60001C4301A80421FFF74DFE00200F21012264
:104B7000FDF71AFB024B1C70201C03B030BDC04671
:104B800023000010F0B583B0FFF7D2FF051CAA0781
:104B900000D587E000200F210122FDF705FB0A2444
:104BA00005E001A80121FFF72DFE013CE4B2002C35
:104BB000F7D100200021FFF715FF0026012862D160
:104BC0000820D5214900FFF70DFF012833D101ACA2
:104BD000201C0421FFF716FEA378012B53D101AB53
:104BE000DB78AA2B0CD04EE0A920311CFFF7FAFE8F
:104BF00000280CD00020391C01F052FB013C04E0DD
:104C0000FA24A4008026F605271C002CECD10026EF
:104C1000002C38D03A20311CFFF7E4FEB04232D1EC
:104C200001AC201C0421FFF7EDFD237804265A0671
:104C300029D50C2627E0A9200021FFF7D3FE012368
:104C400083429B415B420226F61AFA24A400271CE9
:104C50000AE0A9200021FFF7C5FE002806D00020A9
:104C6000391C01F01DFB013C002CF2D1002C09D0B5
:104C7000102080218900FFF7B5FE434243415B428B
:104C80001E4000E00026084B1E70002E02D0FE20C1
:104C9000054002E001200543EDB2044B1D70FFF713
:104CA0005FFE281C03B0F0BDE904001023000010D3
:104CB00070B50D1C161C1C1CFFF73AFF0323C2071E
:104CC00037D40423002C34D01B4B1B781A0700D494
:104CD0007602012C0FD11120311CFFF783FE002832
:104CE00022D1281C80218900FFF7EAFE434243417C
:104CF0005B421C4018E01220311CFFF773FE0028B5
:104D000012D18026B600281C311CFFF7D9FE0028DE
:104D100006D080239B00ED18013CE4B2002CF2D1B8
:104D20000C200021FFF75EFEFFF71AFE631E9C4178
:104D3000E3B2181C70BDC046E9040010F8B50E1CA3
:104D4000171C1D1CFFF7F4FE0324C20741D40224E4
:104D500043073ED40424002D3BD01F4B1B781A0779
:104D600000D47F02012D0ED11820391CFFF73AFE26
:104D7000002829D1301CFE21FFF77CFE434243412D
:104D80005B421D4020E006221A4203D09720291CD6
:104D9000FFF728FE1920391CFFF724FE002813D145
:104DA000301CFC21FFF766FE002806D080239B0004
:104DB000F618013DEDB2002DF2D10020FD21FFF7E4
:104DC00059FE002800D10125FFF7CAFD6C1EA54140
:104DD000ECB2201CF8BDC046E904001070B584B0E8
:104DE0000C1C151CFFF7A4FE031C0320D90750D48C
:104DF000012C0DD0002C02D0032C42D045E0FFF74F
:104E0000D9FD0124002841D0FFF7AAFD00243DE090
:104E100009200021FFF7E6FD0124002836D168466D
:104E20001021FFF74DFE002830D06A4613789B0909
:104E3000012B0AD1527A6E46337A1B02D318013302
:104E40009BB29B022B60002420E05079937ADB090F
:104E5000527A0F210140591803231A405200891831
:104E60006A46147AD2796E46B079A4099200A218E3
:104E700003409B02D2180132CB1F9A402A600024C3
:104E800004E080232B60002400E00424FFF768FD89
:104E9000201C04B070BDC04630B583B01D48FDF77E
:104EA000A1FF0120FBF744FC0128FAD01A4B5878E7
:104EB000996A01F0C5FD6D4607350120FBF738FC06
:104EC000041C002001F088FE002808D0002001F01A
:104ED00089FE28700120291C012201F061FE0120B9
:104EE00001F07AFE002808D0012001F07BFE287036
:104EF0000020291C012201F053FE002CDDD00748C0
:104F0000FDF770FF044B5878596801F099FD03B024
:104F100030BDC04610890000E80B00101C8900005D
:104F2000F0B54F464646C0B489B0041C0F1C8578C6
:104F30003D3D6B425D41002D04D00330804601F0C1
:104F400035FF8146667823781B023343BF4CA3426A
:104F500000D101E300D984E0BD4A934201D100F0C1
:104F60007DFC3ED8BB4A934200D10AE11CD8BA4A24
:104F7000934200D17CE209D8B84A934200D135E18E
:104F8000B74A934200D19DE200F0BBFCB54A934280
:104F900000D1F7E1B44A934200D12CE3B34A9342E3
:104FA00001D000F0AEFC55E2B14A934200D11CE3BF
:104FB00009D8B04A934200D1FBE2AF4A934200D1F4
:104FC000DBE200F09EFCAD4A934200D1DDE0AC4A4A
:104FD000934200D1DDE0AB4A934201D000F091FC56
:104FE000C1E0A94A934200D12AE21CD8A74A9342C1
:104FF00000D108E209D8A64A934200D1D8E1A54AD7
:10500000934200D1E7E100F07CFCA34A934200D137
:1050100009E2A24A934200D1FDE2A14A934201D0A3
:1050200000F06FFCEBE29F4A934200D1BFE009D849
:105030009D4A934200D117E39C4A934200D10AE370
:1050400000F05FFC9A4A934200D15FE3994A934291
:1050500000D10CE3984A934201D000F052FC00F0DA
:1050600004FC964A934200D1C8E040D8944A934247
:1050700000D135E21ED8934A934201D100F027FCBB
:105080000AD8914A934200D178E1904A934201D1E3
:1050900000F009FC00F035FC8D4A934200D12DE26E
:1050A0008C4A934200D1A5E08B4A934201D000F094
:1050B00028FC59E1894A934200D16DE209D8884A17
:1050C000934200D15CE2874A934200D1ECE100F0C8
:1050D00018FC854A934200D1ABE0844A934200D148
:1050E00090E0834A934201D000F00BFCCEE1814A6C
:1050F000934200D125E31BD87F4A934200D10BE2B3
:1051000009D87E4A934200D180E07D4A934200D183
:1051100094E300F0F6FB7B4A934200D1ACE37A4A79
:10512000934200D15CE3794A934200D0E9E303E281
:10513000774A934200D163E308D8764A934200D17C
:1051400025E3754A934200D131E3DAE3734A93428F
:1051500000D165E3724A934200D10AE3714A934257
:1051600000D0CEE368E0002D02D06F4B49461970A5
:105170006D4B18780021002201F044FE01F0CAFEB8
:10518000BFE36A48FEF716FABBE36848FEF732FA57
:10519000B7E3002D02D0664B4A461A70644B18786C
:1051A0000021002201F02EFE01F0B4FEA9E303A9C4
:1051B000604A0B1C31CA31C312CA12C300245E4EAE
:1051C0005A4D5E4F0FE0A20003ABD2583260281C4C
:1051D000FEF73EFA306800F041FD3860281CFEF70B
:1051E00027FA0134A4B2042CEDD98AE34F48FEF724
:1051F0001FFA86E34D48FEF72BFA82E34B48FEF791
:1052000051FA7EE34948FEF769FA7AE34C4D4D4B7B
:105210002B60464C201CFEF745FA17235B422B609F
:10522000201CFEF73FFA484B2B60201CFEF73AFA91
:1052300067E3FEF765F964E3002D00D188E04D4691
:10524000012D00D082E0FEF7F3FA81E0534C00001C
:105250005444000044430000534100004C4100000E
:105260005041000052420000434300005A410000F8
:10527000574300004F4300005243000044440000E5
:105280004944000042440000564700004C470000DB
:1052900042470000464700005347000054470000C3
:1052A0005047000041480000584700005A4700009E
:1052B00052490000574900004D4800004954000081
:1052C00054500000574D0000434D0000524D000067
:1052D0004150000052500000584D00004C53000057
:1052E0004352000041530000565300004554000053
:1052F00054530000435A000041550000545400002C
:105300005A54000043580000415A00005455000010
:10531000505A00004D5A00004F5A0000535A0000E6
:10532000545A0000525A0000780900100C870000FF
:10533000B8040010FC880000C4130010600F0010B7
:1053400094110010B5F7FFFF94110000FEF7F8FA72
:10535000D24B1B68002B03D1D14801F049FDD0E2AC
:10536000D04801F045FDCCE2CF4B18680021002267
:1053700001F048FDCD4801F03BFDC2E2CC4ACA4BEA
:105380001A60BEE2002D02D0CA4B48465860C94B95
:1053900058680021002201F035FD01F0BBFD002D11
:1053A00000D1AEE2C34B5878596801F049FBA8E23E
:1053B000002D02D0BF4B49469962BE4B986A00212E
:1053C000002201F01FFD01F0A5FD002D00D198E2A3
:1053D000FDF748F995E2002D03D02D23B54A4C4640
:1053E000D4542D23B34AD05C0021002201F00AFDE1
:1053F00001F090FD002D00D183E22D23AD4AD05C59
:10540000FDF798F87DE2002D03D02C23A94A4D46E4
:10541000D5542C23A74AD05C0021002201F0F2FCD5
:1054200001F078FD6DE2A34D2424285DFA1E41466B
:1054300001F0B6FB285D9D49022201F0B1FB60E25C
:105440009D4801F0D5FCFDF757F901F0D1FC01F0C2
:1054500061FD56E2002D02D0964B48461872954BDE
:10546000187A0021002201F0CDFC01F053FD48E242
:10547000002D02D08F4B494659728E4B587A00212D
:10548000002201F0BFFC01F045FD3AE2002D02D000
:10549000884B4A46DA60874BD8680021002201F029
:1054A000B1FC01F037FD2CE2002D02D0814B4C46BF
:1054B0001C61804B18690021002201F0A3FC01F05F
:1054C00029FD1EE2002D02D07A4B4D461D75794B09
:1054D000187D0021002201F095FC01F01BFD10E277
:1054E000002D02D0734B48469861724B9869002199
:1054F000002201F087FC01F00DFD02E2002D02D038
:105500006C4B4946D9616B4BD8690021002201F0F0
:1055100079FC01F0FFFCF4E1002D03D02023654A63
:105520004C46D4542023634AD05C0021002201F071
:1055300069FC01F0EFFCE4E1002D03D021235D4A7A
:105540004D46D55421235B4AD05C0021002201F056
:1055500059FC01F0DFFCD4E1002D02D0554B484648
:105560005884544B588C0021002201F04BFC01223E
:10557000524B1A8001F0CEFCC3E1FBF7EFF8C0E11B
:10558000002D00D1BDE14946012902D1FDF7E4FE1D
:10559000B7E1FDF765FFB4E1002D00D1B1E14A4666
:1055A000012A02D1464B1A70ABE10022444B1A701B
:1055B000A7E1444B1B78002B00D0A2E1FFF7A6FA2D
:1055C000002800D19DE103A810213F4AFDF760FDAE
:1055D0003E4803A90A22FCF713F8021E00D190E10D
:1055E0003B483C4901F08AFE8BE138483A49424643
:1055F000FCF732FC85E13548FCF7EEFA81E1002D3D
:1056000002D0364B4C461C70344B187800210022D7
:1056100001F0F8FB75E1404601F08EFB142102F029
:1056200037FB041C2E4860432E4902F031FB8500F5
:1056300028188500281C2B4902F02AFB061C281C70
:10564000284902F025FB009121482749221C331CE0
:1056500001F054FE55E1404601F06EFB021C1C486F
:10566000224901F04BFE4CE1FFF716FC49E14046B0
:1056700001F030FC1E4B18704446023401253AE01C
:10568000002B37D06378002B34D06E1C201C01F027
:1056900021FC174948550234351C2CE06C090010D8
:1056A000288900002C890000C01300100C8700001E
:1056B00019FCFFFFE80B0010308900001E000010ED
:1056C000D3040010D2040010E8810000C8130010B9
:1056D0003D7500004889000020840000A4040010EB
:1056E000F42C0000102700006C8900007C89000069
:1056F000EC08001001342378002BC1D1834B1D60CE
:105700000022834B1A60FDF7C9F9FAE0404601F028
:10571000E1FB4546013501231843C0B27D4C2070A2
:10572000281C01F0D7FB061C794B1D60774B01222A
:105730001A60FDF7B3F9711C201C002201F0F2FB86
:10574000DFE0002D03D02E23734A4C46D4542E2381
:10575000714AD05C0021002201F054FB01F0DAFB19
:10576000002D00D1CDE02E236B4AD05CFAF7F4FE79
:10577000C7E0002D02D0684B4D461D63664B186B89
:105780000021002201F03EFB01F0C4FBB9E0002D36
:1057900003D02F23604A4846D0542F235E4AD05C62
:1057A0000021002201F02EFB01F0B4FBA9E02E2322
:1057B000594AD35C002B00D0A3E0002D05D0494608
:1057C000CAB201200121FCF7EFFC01200121FCF706
:1057D00023FD0021002201F015FB01F09BFB90E06E
:1057E000002D03D03C234C4A4C46D4543C234A4A17
:1057F000D05C0021002201F005FB01F08BFB80E072
:10580000002D03D03423444A4D46D5543423424A14
:10581000D05C0021002201F0F5FA01F07BFB70E082
:10582000002D02D03C4B484698633B4B986B0021BF
:10583000002201F0E7FA01F06DFB62E0002D03D0D9
:105840003D23354A4946D1543D23334AD0560021A1
:10585000002201F0D7FA01F05DFB52E0002D50D09C
:105860004A46D0B2FDF7F2FA4BE0FCF78FFF2B4B24
:1058700018802B48FDF74EFF002D0CD04B46002B17
:1058800002D0012B04D006E0002001F0F1FB02E081
:10589000012001F0EDFB48460021002201F0B2FAA0
:1058A00001F038FB2DE0404601F0EAF9072828D93D
:1058B000404601F0CDF9046801F002FB3A20FDF703
:1058C000BFFB201C01F0FCFA01F024FB19E040466C
:1058D00001F0D6F9102814D9404601F0B9F9051C99
:1058E0004046093001F0B4F9041C2860281C01F07E
:1058F000E7FA3A20FDF7A4FB201C01F0E1FA01F0E1
:1059000009FB09B00CBC90469946F0BD0C0900108B
:10591000C4080010EC080010E80B00105809001033
:105920000C87000038B5002001F056F9002800D19E
:1059300085E0002001F056F9414B1870031C613BD3
:10594000DBB2192B02D820383D4B18703C4B1B782A
:10595000202B74D0DAB2202A04D8082B33D00D2B98
:1059600024D055E02A2B4DD0512B41D0212B4FD1A3
:105970003448FDF737FA2120FDF762FB324A334BFA
:105980001A60334A334B1A600023324C2F4808E028
:105990002268511C216001684D1C05600978117056
:1059A0000133C72BF4DDFDF7F1F848E001F0B2FA5E
:1059B000294C21782948FFF7B3FA2278284B1A702E
:1059C000002323703BE0244B1B78002B37D0013B96
:1059D000DBB2214A13700021204AD1540820FDF780
:1059E0002FFB2020FDF72CFB0820FDF729FB26E0EC
:1059F000194B1B78002B22D1194B19781748FFF748
:105A00008FFA1CE0144B1B78002B01D1FDF7EEF848
:105A10000B4B1878031C203B5F2B10D80E4B1B78C8
:105A2000132B0CD8FDF70CFB0B4A11784B1CDBB287
:105A300013700A4A0248007850540021D15438BDEE
:105A4000F004001084890000ED2B0000EC0400102D
:105A5000000800100C050010F1040010F404001000
:105A6000F204001008B51E2000211E2200F0A8FB41
:105A700008BDC04608B540006038C0B21021002201
:105A800000F09EFB80B208BD38B5FFF7EBFF0024A5
:105A9000054D05E0201CFFF7EDFF6300585301346E
:105AA000072CF7DD38BDC0460016001070B5002485
:105AB0000025002616E044200021152200F080FB7E
:105AC00000201821002200F07BFB36185420002112
:105AD000152200F075FB00201821002200F070FB59
:105AE0002D180134032CE6DDB608034B1E60AD080B
:105AF000024B1D6070BDC046181600101416001031
:105B0000094B5B891B02094A1268D31A084A1360C1
:105B1000084A1268002A06D00121064A1160D917E6
:105B2000054A1360516070470016001014160010EB
:105B3000F01500102C000010F815001000000000F7
:105B400010B50B4B1868C1170A4B9A89002302F055
:105B5000DCF84C02C20D2243CB15044902488018E0
:105B6000594110BDC046C046D007000000000000EB
:105B7000F015001000160010F8B55F4656464D4669
:105B80004446F0B42D4B1B78012B14D12C490A68E4
:105B90002C4B1B68D3180B602B498B4202D80A2070
:105BA0002849086029498B4203D90A214942254BDB
:105BB0001960101C3BE0264B19688946254B1C6870
:105BC0005D68254B5A88924699888846DA889346BC
:105BD0001A89201C291C002302F097F88B068609DD
:105BE0001E438F114146CB0B4A04B6185F41201C5F
:105BF000291C5A46002302F088F84C06C2092243A9
:105C0000CB110024002551460C0412196B41484663
:105C1000002102F07AF8CC02420D22434B15141CED
:105C20001D1CA41BBD416A04E40B101C20433CBC9A
:105C300090469946A246AB46F8BDC046780900108A
:105C40003400001028000010E7030000C0D4010059
:105C500018160010F81500100016001008B50E4BAD
:105C60001B78022B13D10D4A10680D4B1B68C3180B
:105C700013600C4A934203DD39214942084A1160FE
:105C8000094A934206DA3922054B1A6002E00021E4
:105C900001F0E8F908BDC046780900103000001096
:105CA00024000010289A010030F8FFFF08B5EC200E
:105CB0001E21FCF71DFF08BD10B582B04100603900
:105CC000C9B2EC20FCF714FF6C460634EC20211C12
:105CD0000222FCF72DFF201C022101F001F920888F
:105CE00002B010BDF8B5FFF7E1FF0024064E074FE4
:105CF00006E06500AF53201CFFF7DEFFA853013418
:105D0000072CF6DDF8BDC046001600100F27000076
:105D1000F0B5474680B482B000230193009300247D
:105D200000250026FA239B0098461F4F32E040468C
:105D300000F09AFAEC204221FCF7DAFE381C00F061
:105D400093FAEC200021FCF7D3FEEC2001A90322FA
:105D5000FCF7EEFE01A8032101F0C2F8019BF61842
:105D6000404600F081FAEC205221FCF7C1FE381CBD
:105D700000F07AFAEC200021FCF7BAFEEC2069462C
:105D80000322FCF7D5FE6846032101F0A9F8009B29
:105D9000ED180134002CCADD044B1E60044B1D605D
:105DA00002B004BC9046F0BDE204000018160010DA
:105DB0001416001010B5CF4B1B78DBB20A2B00D99C
:105DC000BDE19B00CC4AD3589F46CC4B1B68022BAD
:105DD00011D0042B1DD0012B00D0B0E10122C74B04
:105DE0001A6001200521FCF7DFF9012005210022BE
:105DF000FCF79AF9A3E10222C04B1A6001200521A9
:105E0000FCF70AFA002800D099E10122BC4B1A7075
:105E100095E1BA4B04221A6002225A6000225A61AC
:105E20000122B44B1A708AE1B44B1B68022B15D0C7
:105E3000042B1CD0012B00D081E1B04A1360B14A81
:105E40001278B1490978D2B20A41134200D176E101
:105E5000012005210122FCF7A7F970E10222A74BDE
:105E60001A60012005210122FCF79EF967E1042256
:105E7000A24B1A60A44B1A780132D2B21A701B7866
:105E8000082B24D10022A04B1A70A04B1A88013293
:105E900092B21A801A889E4B1B8892B29A420DD1F8
:105EA0000322944B1A70012005210022FCF73CF9D3
:105EB000924B02225A6000225A6140E1934B1B88A8
:105EC000944A1268D3181A78D2B28E4B1A708B4C3F
:105ED00002236360012005210122FCF725F901203E
:105EE00005210022FCF760F90123636027E1834B61
:105EF0001B68022B11D0042B24D0012B00D01EE1F3
:105F000001227E4B1A6001200521FCF74DF901208A
:105F100005210022FCF708F911E10222774B1A60F3
:105F200001200521FCF778F9002800D107E1764B24
:105F30001B78DBB201229A40724B19780A43D2B225
:105F40001A70FCE004226D4B1A606F4B1A78013214
:105F5000D2B21A701B78082B1FD16C4B1A886D496E
:105F600009688A1867490878C0B2107000220A7060
:105F700065490A701A88013292B21A801A88644BF5
:105F80001B8892B29A4208D105225A4B1A705B4B79
:105F900002225A6000225A61D1E0584C0223636009
:105FA000012005210122FCF7BFF801200521002274
:105FB000FCF7FAF801236360C1E0504B1B68022B29
:105FC00011D0042B18D0012B00D0B8E001224B4B8C
:105FD0001A60514B1B78002B00D1B0E00120052145
:105FE000FCF7E2F8ABE00222444B1A6001200521E5
:105FF0000122FCF7D9F8A2E0404C042323600722D9
:106000003C4B1A70012005210022FCF78DF8022379
:1060100063600023636192E0384B1B68022B11D050
:10602000042B1CD0012B00D089E00122334B1A60D5
:1060300001200521FCF7B8F8012005210022FCF71A
:1060400073F87CE002222D4B1A6001200521FCF739
:10605000E3F8002873D001222F4B1A706FE0274B12
:1060600004221A600921234A117002225A60002278
:106070005A6164E0214B1B68022B10D0042B2BD0FB
:10608000012B5CD101221D4B1A6001200521FCF778
:106090008BF8012005210022FCF746F84FE0022290
:1060A000164B1A6001200521FCF7B6F8002809D02C
:1060B0001A4B1B78012B42D1184B1A780132D2B2FD
:1060C0001A703CE0154B1B78002B38D1134B1A7813
:1060D0000132D2B21A7032E00422084B1A600F4B20
:1060E0001B78022B1CD10B22024B1A700222034B8D
:1060F0005A6024E010050010908900000040014023
:106100001E0500101F0500102005001018050010C6
:106110001C05001014050010110500101A050010D0
:10612000074C02236360012005210122FBF7FCFFDD
:10613000012005210022FCF737F80123636010BD20
:1061400000400140064B0122DA61196819680131EB
:106150005960044B1A70044B1A6801321A60704778
:10616000000005401C1600102016001008B5002085
:1061700016210122FBF7D8FF00200F210122FBF797
:10618000D3FF00200E210122FBF7CEFF00201021BB
:106190000022FBF7C9FF002011210122FBF7C4FFF9
:1061A000002016210122FBF7FFFF00200F21012212
:1061B000FBF7FAFF00200E210022FBF7F5FF08BDD8
:1061C000F8B5051C0E1C171C002016210022FBF739
:1061D000EBFF002417E0EA0900201121FBF7E4FFA0
:1061E0006D00EDB200200E210122FBF7DDFF002340
:1061F00001E0C0460133092BFBDD00200E21002207
:10620000FBF7D2FF0134072CE5DD0020112100222D
:10621000FBF7CAFF0025002416E06D0000200E21C8
:106220000122FBF7C1FF002301E0C0460133092B27
:10623000FBDD00201021FBF7EFFF054300200E21BE
:106240000022FBF7B1FF0134A642E6DC002F03D0A9
:106250000020391C00F024F8002016210122FBF751
:10626000A3FF281CF8BDC046002315E0C046C04669
:10627000C046C046C046C046C046C046C046C046EE
:10628000C046C046C046C046C046C046C046C046DE
:10629000C046C04601339BB28342E7D37047C04635
:1062A00038B50D1C00281BD11C4C02236360002351
:1062B000E3601B4B996F1B4B186801F0ECFC1A490B
:1062C00001F0E9FC4543A561FF23236004236361DA
:1062D00001236360211C01224B681A42FCD11CE09F
:1062E00001281AD1114C022363600023E3600C4B98
:1062F000996F0C4B186801F0CEFC0B4901F0CBFCF8
:106300004543A561FF232360042363610123636088
:10631000211C01224B681A42FCD138BD008001408B
:1063200000800440880400101027000000C00140D5
:1063300038B50D1C002818D1194C022363600023C6
:10634000E360184B1868FA21890001F0A4FC45436A
:10635000A561FF2323600423636101236360211C83
:1063600001224B681A42FCD119E0012817D10E4CCA
:10637000022363600023E3600A4B1868FA21890056
:1063800001F089FC4543A561FF2323600423636179
:1063900001236360211C01224B681A42FCD138BDE5
:1063A000008001408804001000C001402C4B1B6895
:1063B000DA0706D501222A4B1A602A4B1A680132E5
:1063C0001A60274B1B689A0706D50222244B1A60D5
:1063D000244B5A6801325A60214B1B685A0706D574
:1063E00004221F4B1A601F4B9A6801329A601C4BA3
:1063F0001B681A0706D50822194B1A60194BDA6870
:106400000132DA60164B1B68DA0606D51022144BEF
:106410001A60154B1A6801321A60114B1B689A06F4
:1064200006D520220E4B1A600F4B5A6801325A6073
:106430000B4B1B685A0606D54022094B1A600A4BC3
:106440009A6801329A60064B1B681A0606D58022AC
:10645000034B1A60044BDA680132DA607047C046B9
:106460000080014024050010340500102C4B1B68EF
:10647000DA0706D501222A4B1A602A4B1A68013224
:106480001A60274B1B689A0706D50222244B1A6014
:10649000244B5A6801325A60214B1B685A0706D5B3
:1064A00004221F4B1A601F4B9A6801329A601C4BE2
:1064B0001B681A0706D50822194B1A60194BDA68AF
:1064C0000132DA60164B1B68DA0606D51022144B2F
:1064D0001A60154B1A6801321A60114B1B689A0634
:1064E00006D520220E4B1A600F4B5A6801325A60B3
:1064F0000B4B1B685A0606D54022094B1A600A4B03
:106500009A6801329A60064B1B681A0606D58022EB
:10651000034B1A60044BDA680132DA607047C046F8
:1065200000C001404405001054050010002803D1AC
:106530000122034B5A6002E00122014B5A6070476E
:106540000080014010B500285FD100291BD1594BB4
:106550009A6C07218A439A64986C032210439864CA
:10656000D86C8843D864D86C1043D864586D88437D
:106570005865586D10435865986D88439865996DB6
:106580000A439A6594E001291CD14A4BB0201A585D
:1065900007218A431A501C58032214431C50986840
:1065A00088439860986810439860D8688843D8609A
:1065B000D8681043D86018698843186119690A437C
:1065C0001A6175E002291FD13A4B802299580720A1
:1065D000814399509C5802210C439C5084229C5822
:1065E00084439C509C580C439C5088229C58844364
:1065F0009C509C580C439C508C229C5884439C502B
:1066000098580143995053E0FEE700291BD1294BCC
:106610001A6E07218A431A66186E03221043186601
:10662000586E88435866586E10435866986E884373
:106630009866986E10439866D86E8843D866D96E6F
:106640000A43DA6634E001290FD11A4B9A6907210F
:106650008A439A619869032210439861D8698843F4
:10666000D861D9690A43DA6122E002291FD1114BAE
:10667000E02299580720814399509C5802210C43ED
:106680009C50E4229C5884439C509C580C439C5042
:10669000E8229C5884439C509C580C439C50EC220C
:1066A0009C5884439C5098580143995000E0FEE761
:1066B00010BDC0460040044070B5141C002825D110
:1066C000264B5D6840222A435A6080229E588025CE
:1066D000AD0035439D50FFF735FF0023204D0022CC
:1066E000204803E099004A510A500133032BF9D99D
:1066F0001D4B9C61DC611C625C621C4A9A621C4AF4
:106700005A61802212021B4B1A6025E0012823D116
:10671000124B5D68802215435D609E588025ED0018
:1067200035439D50FFF70EFF0023134D0021134802
:1067300003E09A00515111500133032BF9D9104B4A
:106740009C61DC611C625C62084A9A62084A5A6178
:1067500080225202074B1A6070BDC0460080044080
:106760002405001034050010008001406D0B00006E
:10677000DB06000000E100E04405001054050010B5
:1067800000C0014043011B18DB00154AD318013338
:10679000FF335A799B79D2B29A420FD3104B420100
:1067A0001118C90059180131FF3149791218D20066
:1067B0009B180133FF339B79C81A10E0084B420144
:1067C0001118C90059180131FF3149791218D20046
:1067D0009B180133FF339B79C81A0130FF30704793
:1067E0002416001070B5041C0E1CFFF7CBFFFE280A
:1067F00012DC0A4B62011519ED005D190135FF35F8
:106800006879C0B2411CC9B269711119C900081870
:10681000181846712B1C5B7970BDC04624160010F9
:1068200038B5041CFFF7AEFF002818DD0D4B6201E0
:106830001019C00018180130FF308179C9B24D1C01
:10684000EDB285711019C000411859184879C0B2CD
:106850001419E4001B190133FF339B7900E0002079
:1068600038BDC0462416001008B51D4B9B681B0799
:106870005B0F032B14D11A4B5B69FF2213409E223E
:106880001A4204D0174A1360154B1B6827E0DA0739
:1068900025D5134B1968C9B20020FFF7A3FF1EE0EE
:1068A000022B06D10E4B1968C9B20020FFF79AFFE0
:1068B00015E0062B06D10B4B1968802252000A43C3
:1068C0001A600CE0012B0AD1054B5B699A0603D5CF
:1068D0000122044B1A7102E00022024B1A7108BD1A
:1068E000008000402416001008B5214B9B681B0750
:1068F0005B0F032B16D11E4B5B69FF2213409E22B8
:106900001A4206D0842252001A498B50184B1B6839
:106910002DE0DA072BD5164B1968C9B20120FFF715
:1069200061FF24E0022B06D1114B1968C9B2012086
:10693000FFF758FF1BE0062B08D10E4A84235B00AB
:10694000D058802149000143D15010E0012B0ED1D5
:10695000074B5B699A0605D5012186235B00054A32
:10696000D15404E0002186235B00024AD15408BDC3
:1069700000C000402416001010B5002823D10029C3
:106980000FD12E4B9A6C07218A439A64986C02228D
:1069900010439864D86C8843D864D96C0A43DA648D
:1069A0004AE0012948D1254B5A6F07218A435A678B
:1069B000586F042210435867986F88439867996FFF
:1069C0000A439A6738E0012835D100290FD11B4BC3
:1069D0009A6E07218A439A66986E0222104398663F
:1069E000D86E8843D866D96E0A43DA6624E0012956
:1069F00011D1124BEC2299580720814399509C5891
:106A000005210C439C50E8229C5884439C50985884
:106A10000143995010E0094BDA6A07218A43DA6290
:106A2000D86A03221043D862186B88431863196B25
:106A30000A431A6300E0FEE710BDC0460040044070
:106A4000F8B50F1C43011B18DB004F4AD318012275
:106A50001A710133FF3300225A719A7100234A4E92
:106A600045012D18ED00002403E0EA18B218547116
:106A70000133FF2BF9D9002842D180248022D20291
:106A8000424B1A510021FFF777FF414B596804220E
:106A90000A435A601959802252010A431A51982216
:106AA000012199503B4C8321E16099583A4B186879
:106AB00001F0F1F80009391C01F0EDF8030A6360F8
:106AC000FF23184020600323E3601023A362072301
:106AD000A3606369211C60224B691340602BFBD1CA
:106AE00001E01A6801E02B4B01215A691142F8D1EB
:106AF0008022D202254B1A600522264B5A6041E0C3
:106B0000802480221203214B1A510021FFF734FF09
:106B10001F4B596808220A435A6019598022920172
:106B20000A431A519C22012199501C4C8321E16097
:106B30009958194B186801F0AEF80009391C01F09A
:106B4000AAF8030A6360FF23184020600323E36070
:106B50001023A3620723A3606369211C60224B6991
:106B60001340602BFBD101E01A6801E00B4B0121BF
:106B70005A691142F8D180221203044B1A6005228F
:106B8000064B5A60F8BDC0462416001000E100E034
:106B900000800440008000408804001000C00040D5
:106BA00070B50B4E20230B4D0EE0002805D16C690B
:106BB0002342FCD00C782C6004E074692342FCD0A2
:106BC0000C7834600131013A002AEED170BDC04624
:106BD00000C000400080004008B5FFF7D3FD431E11
:106BE000984108BD10B5041CFFF7CCFD031C002024
:106BF000002B02D0201CFFF713FE10BD031C021C4B
:106C0000303AD2B2101E09280DD91A1C613A052A51
:106C100002D8573BD8B206E000201A1C413A052A98
:106C200001D8373BD8B27047F8B5071C00230024C1
:106C30004E0006E01D01FFF7E1FF031C2B4301346A
:106C4000E4B2B44202DA385D0028F3D1181CF8BD72
:106C500008B50421FFF7E8FF08BDC04603E09342F2
:106C600009D1013001310378002B06D00A78002ABF
:106C7000F5D1002002E0012000E000207047C0466E
:106C8000021C002001E0013080B2135C002BFAD11D
:106C90007047C046F0B557464E464546E0B4051C21
:106CA0000F1C002808D1002903D13020FCF7C8F9B7
:106CB0003BE030230B7038E00026002809DA002979
:106CC00003D12D20FCF7BCF902E02D230B70012627
:106CD0006D4201239946174C00239A461EE0A846B0
:106CE000281C211C00F0D7FF051E02D14B46002BAB
:106CF0000CD1281C3030C0B2002F03D1FCF7A0F912
:106D0000D14603E0731CB855DEB2D1466543434615
:106D10005D1B201C0A2100F0BEFF041C002CDED1EC
:106D2000002F02D0BE19002333701CBC9046994638
:106D3000A246F0BD00CA9A3B30B500E001300378AE
:106D4000002B05D01A1C303A092A01D92D2BF5D178
:106D500001252D2B01D101306D42002305E0990062
:106D6000CB185B00303AD31801300278111C30394F
:106D70000929F4D92E2A11D1013000220BE0990003
:106D8000CB1859000B1C0478002C03D0231C303B7B
:106D9000CB1801300132032AF1DD01E0024A5343EE
:106DA000281C584330BDC0461027000010B500E035
:106DB00001300378002B05D01A1C303A092A01D97A
:106DC0002D2BF5D12D3B5A4253415B4201221343F7
:106DD000002205E09400A218520030398A180130D0
:106DE00001780C1C303C092CF4D9181C504310BD00
:106DF00010B5041C02E0FCF723F9013420780028C8
:106E0000F9D110BDF0B5474680B40D1C161E0C2EEE
:106E100000D90C260023002E07D1291CFFF73AFFCA
:106E20002FE0E1540133DBB201E0174C00210C2BC1
:106E3000F7D91549FFF72EFF711E134ECBB29846B6
:106E4000301CB446202709E0434603E05A1E845C08
:106E5000C454D3B2002BF9D163461F70735C002B6E
:106E6000F2D00023002D04D108E0EA540133DBB254
:106E700000E00549CA5C002AF7D102E00248FFF7AA
:106E8000B7FF04BC9046F0BD6405001038B5051C82
:106E90000309054CE05CFCF7D3F80F231D40605D4F
:106EA000FCF7CEF838BDC046308A000010B5041C8F
:106EB000000AFFF7EBFFE0B2FFF7E8FF10BDC046A6
:106EC00010B5041C000CFFF7F1FFA0B2FFF7EEFFB6
:106ED00010BDC04608B50121FFF7A6FEC0B208BD2F
:106EE000032908D004290BD0022911D10378427854
:106EF000027043700CE0037882780270837007E0C0
:106F00000378C2780270C3704378827842708370CD
:106F10007047C04608B50D20FCF792F80A20FCF730
:106F20008FF808BDF8B557464E46C0B4071C0E1C76
:106F30009246002A06D01748FFF75AFF00240F2375
:106F400099461CE01448FFF753FFF7E74B462342EE
:106F50000ED1FFF7DFFF5346002B03D07819FFF760
:106F6000AFFF02E0A0B2FFF7A1FF0C48FFF740FF20
:106F7000785DFFF78BFF2020FCF762F80134251EB7
:106F8000B542E3D3FFF7C6FFFFF7C4FF0CBC914641
:106F90009A46F8BDBC890000F88900001482000000
:106FA00070B50E1C151CFFF723FF002406E0305DB2
:106FB000FFF76CFF2020FCF743F80134AC42F6D316
:106FC000FFF7A8FF70BDC046031C00208B4203DB07
:106FD000D80FD1179A4248417047C046F8B54F467E
:106FE0004646C0B481461C4B1B68834202DD1A4BE7
:106FF00058682CE08923DB00174AD35800248342C9
:1070000021DA164BD05822E0E300DE59651CEB0074
:10701000DA5990464846311CFFF7D6FF002810D0B9
:107020004346991B0C4BE4001C196468ED005B1986
:107030005868001B4A46961B704300F029FE201832
:1070400005E02C1C00E0044F882CDDDD00200CBC8A
:1070500090469946F8BDC046380000104C04000028
:107060007047C04608B5FFF7B9FFFFF7F9FF08BD45
:1070700030B51B4B00221A628E2189005C582025F6
:10708000AC435C501A62002301E0C0460133C72BB9
:10709000FBD9134B186401225A64002159645A64C5
:1070A000191C4B6C1A42FCD00D4B41229A608E2267
:1070B00092009958802081439950191C0122CB6875
:1070C0001A42FCD0064B03221A6701225A6700219C
:1070D00059675A67191C4B6F1A42FCD030BDC04625
:1070E000008004401F4B022210B51F491A601F4A3E
:1070F0002024D16700228E211A6289005858A043AB
:1071000058501A62C822C046013A002AFBD1012118
:107110001A6459645A645964596C124AC807FBD5F9
:10712000412191608E21890050588024A043505005
:10713000D86801210B4A0842FAD0032010670020CA
:10714000516750675167596F01221142FBD0054BBF
:107150009A67074A00231360064A1360064A1360C1
:1071600010BDC046008004401F00010004800440A0
:1071700094800440988004409C800440F0B5071C33
:1071800089B00D1C141C00262B78002B00D1B0E018
:10719000252B00D0A8E06A786B1C002A00D1A8E05B
:1071A000252A00D19FE0002005902D2A02D101213F
:1071B000AB1C05911D1C2A786B1C302A05D1059A41
:1071C0001D1C02231A430592F5E70421101C884375
:1071D0002A2802D10022101C08E0303A092AF9D9E5
:1071E000002216E02E2908D1012001335D1E2978E6
:1071F0002A29F7D122680434F7E730390491C9B25B
:10720000092906D80028F0D10A256A4304995218A2
:10721000EBE72B786C3B59424B41ED182B78702BE8
:1072200032D00CD8632B4DD0642B15D0582B55D1B0
:10723000211D049121680092059A019231E0752B7D
:1072400035D0782B18D0732B48D12168231D049397
:1072500000293ED128493CE021680092059A201D72
:107260006123049001920293381C0A22012300F04A
:107270008EF83618049C3AE00598231D2168049383
:107280000092019061230DE03020B8477820B84784
:10729000231D0493059808232168009302230343C8
:1072A000019341230293381C10220023DFE7211DA4
:1072B000049121680092059A612301920293381C7F
:1072C0000A22F2E7231D0493236807A90B70002309
:1072D0004B70381C059B00F01DF8CAE72520B84705
:1072E0002878B84703E01D1C2878B84701360135D7
:1072F0004AE7301C09B0F0BD448A00000EB403B563
:1073000003AA08CA191C0192FFF738FF02B008BC93
:1073100003B01847F7B5141C00900191002A0FDD47
:107320000A1C0199501A1178002901D00132F8E79E
:10733000A04201DA241A00E00C1C30259A0700D480
:1073400020250026D9070BD4261C002E04DDE8B228
:10735000009A9047013EF8E7E643F6172640A41B43
:10736000371C01998B1BD85D002803D0009B9847E0
:107370000137F6E7261C002E04DDE8B2009A90479C
:10738000013EF8E7E043C01704403819FEBDF0B5F0
:1073900087B0071C00920C1E09D103AB30221A7073
:1073A00059700C9A191C0D9BFFF7B4FF40E00022A6
:1073B0000192934207D0009B0A2B04D1914202DA3A
:1073C00001224C42019200226B466E46DA75163657
:1073D000751C002C11D0201C009900F05CFC0929C0
:1073E00002DD0E9B3A3BC91830313170201C0099E8
:1073F00000F051FC013E041CEAE7019B002B10D079
:107400000C9A002A09D00D9B9B0706D52D20B84762
:107410000C9A0124013A0C9203E0013D2D232B70BC
:107420000024381C291C0C9A0D9BFFF773FF2018B1
:1074300007B0F0BD08B50020011C021C00F008F8E0
:10744000FCF790FA08BD08B500F076FC08BD000016
:1074500070B5244CA02200215200201C00F0B2F88C
:10746000C02000F083FA204D0021C022286000F0E7
:10747000A9F828680023282218215A435943A21842
:10748000411801335162082BF5D1221C1749002005
:1074900000F068F9802280235B01201C0021D200CB
:1074A00000F028F8261C124D2836291C321C012019
:1074B00000F058F980228023301C5B0150340021F9
:1074C000D20000F017F8291C221C022000F04AF913
:1074D00080228023201C0021D2005B0100F00AF8EA
:1074E00070BDC04638180010341800104B8A0000D8
:1074F0004D8A0000F0B5C5680124AE071AD0802679
:10750000B600B2420BD08026F600B24204D08026EC
:10751000A640B2420ED102E0416A231C04E0064EAE
:107520005F1E0124B74205D82A4301610160C3618F
:10753000C2600024201CF0BDFEFFFF00084908B512
:107540000B6B013B0B63002B05DB8B6A5A1C8A62B9
:107550001870C0B202E0283100F05AF808BDC046E9
:107560003818001010B5021C1378002B01D001321E
:10757000FAE7CC5CD4540133002CFAD110BD0000E2
:10758000031C0B4330B59A0711D1021C0B680B4C3E
:107590001D190B4C9D43254202D108C20431F5E769
:1075A000D9B211700132002907D01B12F8E700236D
:1075B000CA5CC2540133002AFAD130BDFFFEFEFE80
:1075C0008080808008B500F0CDFB08BDC268202314
:1075D0009A43436A10B5041CE2605B6882699A4270
:1075E0000DD000F0F3F8E268074B1340102213436C
:1075F000626AE3605368A361236993602360E26871
:10760000024B1340E36010BDEFCFFFFFBFBFFFFF92
:10761000F8B5514ACB68061C1A400C1CCA60980683
:1076200002D5081CFFF7D2FFA268E368511C0EDAEE
:1076300098050CD4022149428A1AA2609022520273
:107640001343E36023685A1C22601E7081E0434AA2
:107650001D1C1A40022A05D00022A260802213437A
:10766000E36054E03E490B40802109028B420AD17D
:107670000021201C00F0DCF9E168890602D5201CFD
:10768000FFF7A4FFE56890235B02F0222B43120171
:10769000E36015421ED1606900F080FB00280BD02A
:1076A0006A0509D5636A236123600123E36192239C
:1076B0005B022B43E3600DE080277F01381C00F064
:1076C00055F99423E2685B022B431A432061206042
:1076D000E761E26090210901226825690B4219D017
:1076E000636A99688A4200D9111C491B09D1636AEF
:1076F0006A1C9A602260E269511EA160DA602E70F5
:1077000027E0281C221C00F093F80028EFD001206D
:1077100040421FE0511CF0B221601070626A27687D
:10772000916884468F4200D9391CE769491BD760AC
:10773000580504D463460A2B01D0B94209DB002363
:107740009560281C2560A360221C00F071F80028B9
:10775000DDD1F0B2F8BDC046FFFFF7FF8A10000090
:1077600010A0000070B50D1C061C101C141C00F0AD
:107770000DF92B78722B06D0772B07D0612B20D1F7
:107780000823114A04E00023012201E0042302221D
:10779000013529782B2905D0622908D104210A4313
:1077A000012102E003210A4302210B43F0E7E260DA
:1077B00066611A0706D5201C0021022200F038F964
:1077C00000E00024201C70BD0280000038B5436A30
:1077D000041C056902689968C36813481840E06092
:1077E00082201840022802D0012040421AE0802066
:1077F0004002184016D0914200D2111CA94209D172
:10780000636AE2689D60094B002013402560A06018
:10781000E36007E0491B281C221C00F009F800283F
:10782000EED0E1E738BDC046FFFFF7FFFFFFFEFFE8
:10783000F7B5D56801900E1C141C5769EA0205D5EE
:107840001023381C1D4300F0A6FAA061114B1D4205
:1078500008D0381CA16900F0A7FA002813DB0E4BF2
:107860001D40E560321C381C019900F0A3FA801B12
:10787000431E9841404243005B08F61AA3699E19D3
:10788000A661002805D0E268802313430120E3604D
:107890004042FEBD10000200EFFFFDFFF8B52E4F85
:1078A000C51C3C68AD08002819D0002610E02168EE
:1078B00080228C46A368520591423ED119686268C5
:1078C00061450ED159689B68521803326260A3600B
:1078D000002CECD10C3000F081F9421C30D100209A
:1078E00039E0AA4206DBE91C914203DB80239B05B9
:1078F000236020E0291C0A318A4210D980218905A1
:10790000201C21600C30A90041186560A160521B49
:1079100080246405033A0C604A608B601BE0002BF6
:107920000BD19200801A00F059F90130D7D0802392
:107930009B0523606560201C0CE0261C1C1CC7E70F
:1079400080239B05036045608460002E01D1386070
:1079500000E0B0600C30F8BD78190010002803D0AA
:1079600080230C385B0503607047000010B5FFF7FB
:1079700095FF041E05D10449172200F01BFA00F000
:1079800006FA201C10BDC0464F8A0000F0B5436ABD
:10799000C56889B0041C476906690193AB0726D006
:1079A0002B0716D400F02AF8381C00F0F1F92B054B
:1079B00002D5301CFFF7D2FF0F4BAD0DAD059D4238
:1079C00007D103A8216A142200F0F1F903A800F0FE
:1079D000D1F800211822606AFFF7F4FD201C002175
:1079E0002822FFF7EFFD019B0020636201E00120E8
:1079F000404209B0F0BDC046000080AD38B5002857
:107A000003D000F00BF9051C0EE0041C051C074810
:107A1000201800F003F9002801D001256D42A023B1
:107A200028345B009C42F2D1281C38BD3818001065
:107A3000F7B53B4B0D1CC168041C161C476900912F
:107A4000194269D0381C00F0A9F90190002863D1CF
:107A5000012E04D0022E07D0002E5DD123E0201C81
:107A600000F062F82D181EE0381C00F094F9E1686F
:107A7000002804DA80231943E16001264DE0626AA0
:107A8000266893689E4200D9331CA6699B19266913
:107A90009B1B8E0603D55268934200DA131C834267
:107AA00000DA031CED18002D36DB009E636AB60475
:107AB00004D522689968914200D29A60A1698D42EA
:107AC0000DDB20689A68824200D2021C2069561899
:107AD000361AB54203DCDF68CE19B54207DB009EDB
:107AE00000212022A160616032435D6010E0009EB1
:107AF0006D1AB60701D5EF1BA760009EF60702D5E9
:107B0000821AAA186260009A4519202325609A43B8
:107B1000044B1A40E26001E0022601960198FEBD86
:107B200003001000BFCFF7FFC368990705D1104BC2
:107B3000212201201A60404218E0202219030BD5AF
:107B4000134202D0436A586804E0036881695A18F6
:107B50000369D01A013809E0134202D0436A586819
:107B600004E0036881695A180369D01A7047C04657
:107B70007405001010B5041C00F006F8011C201C50
:107B800000F00FF910BD000010B5411C820706D0AF
:107B90000130431E1B78002BF8D1401A18E003680F
:107BA0000C4A9C180C4A9C43144201D10430F6E75D
:107BB000DCB2421C002C0AD0FF242402821C234287
:107BC00005D0FF242404C21C234200D0021D501AF9
:107BD00010BDC046FFFEFEFE8080808070B50C4C5C
:107BE0002368002B01D10B4B2360C61C256803239F
:107BF0009E43AE19301C00F035F8002802D12660F3
:107C0000281C04E0044B0C2201201A60404270BD85
:107C10007C1900108019001074050010C36870B53D
:107C2000041C032018401AD09A0605D5636A201C4C
:107C30005D68FFF7CBFC04E02368A2699D18236907
:107C4000ED1AE268064B201C1340E360FFF7BEFD0F
:107C5000291C061C0022201CFFF7EAFE301C70BD08
:107C6000FFCFFFFF084B6A469A4202D90123904298
:107C700007D2064B002B01D1002302E09842FBD330
:107C80000123181C7047C046801900100000000036
:107C900003000B4321D4002931D00122D20703096C
:107CA00001E0090112099942FBD9430801E04900AA
:107CB00052089942FBD900E04908401A07D35241C3
:107CC000FAD301461046704749084018F7D2921877
:107CD000FAD34018014610467047CB0F00D04942F6
:107CE000021000D54042534008B5FFF7D4FF0CBC4A
:107CF000521000D34042002A00D549421847F446AA
:107D0000002000F001F86047704710B5434351432D
:107D1000C918040C130C5C43091992B2040C5443A7
:107D200080B2434350432204240C801861411A045A
:107D30001B0C8018594110BD8446830708D18B075E
:107D400006D1131F04D304C904C0043BFBD21A1D7F
:107D5000524205D0891A801A8B5C83540132FBD1C0
:107D6000604670478446043A09D3830707D1090661
:107D70000B0A19430B0C1943043A02C0FCD204321B
:107D800003D001700130013AFBD160467047FEE735
:107D9000012040427047012040427047012040428C
:107DA0007047012040427047012040427047012047
:107DB00040427047101C7047D01F0000AA1F0000EF
:107DC000BC1F0000C41F0000C41F0000C41F00002F
:107DD000C41F0000C41F0000C41F0000C41F000017
:107DE000C41F0000C41F0000C41F0000D41F0000F7
:107DF000C41F0000C41F0000C41F0000261F000095
:107E0000C41F0000BC1F0000C41F0000C41F0000EE
:107E1000C01F0000222A2B2C3A3B3C3D3E3F5B5DBD
:107E20007C7F0000EBFE904D53444F53352E3000C5
:107E30004E4F204E414D45202020204641543332A4
:107E4000202020004E4F204E414D4520202020462E
:107E50004154202020202000726D632E44617465FF
:107E60003A2025640D0A000024206E6F7420666F8E
:107E7000756E642E20626164206D65737361676541
:107E80002E0D0A004D657373616765206368656335
:107E90006B73756D205B253032585D20213D20636A
:107EA000616C63756C6174656420636865636B7392
:107EB000756D205B253032585D2E0D0A00000000E4
:107EC000504D544B0000000047474100524D4300C5
:107ED0002C200000556E6B6E6F776E0024504D5451
:107EE0004B3630352A33310D0A000000436F6D6D7B
:107EF000204572726F720000262800009029000051
:107F0000902900009029000090290000902900008D
:107F100090290000902900004A28000090290000C4
:107F2000902900009029000090290000902900006D
:107F3000902900009029000070280000902900007E
:107F4000902900009029000090290000902900004D
:107F5000902900009029000080290000902900004D
:107F6000902900009029000090290000902900002D
:107F700090290000902900009C2800009029000012
:107F8000902900009029000090290000902900000D
:107F900090290000902900009C28000090290000F2
:107FA00090290000902900009029000090290000ED
:107FB00090290000902900009029000090290000DD
:107FC00090290000902900009029000090290000CD
:107FD0009029000090290000F4280000902900005A
:107FE00090290000902900009029000090290000AD
:107FF00090290000902900008029000090290000AD
:10800000902900009029000090290000902900008C
:1080100090290000902900001829000090290000F4
:10802000902900009029000090290000902900006C
:1080300090290000902900005C2900006977623ACD
:108040002000000069773A20000000006972623A5F
:108050002000000069723A2000000000E02F0000BC
:108060006E2E0000B22E0000D02E0000322F000035
:10807000922F000000000100020004000800100020
:1080800020004000800000010002000400080010F1
:10809000002000400080030006000C0018003000A3
:1080A000210000030006000C001800304020C00032
:1080B0008001FF3F00000011220049046D15E42EED
:1080C000892A0001000A8020C03F4015002040049A
:1080D000004000223F2206005B044F0466046D044A
:1080E0007D0407007F046F0409000A00000A4104B0
:1080F000802003147F1577040F1539000F117904C0
:1081000071043D04760409111E00700A3800B6029D
:10811000B6083F0073043F08730C6D0401113E0064
:1081200030223628802A62144926390080080F0040
:1081300023000800800058087C0458045E0458207E
:1081400001150C0C740400101021001B00115414B4
:1081500054045C04031561090014080C40151C004C
:1081600004081C10402C80124820400A0011802472
:108170005204082800010203020105040405060751
:1081800007060300010101000000010100000000DA
:1081900001010100383E00004E3E0000643E000038
:1081A000A23E0000CE3E0000123F0000423F000011
:1081B000703F0000AA3F0000E63F00000E400000B4
:1081C0003A4000004572726F72206D6F756E74696F
:1081D0006E672064726976652E0D0A00434647205B
:1081E0005265616400000000303A73746172747506
:1081F000702E74787400000025730D0A00000000D2
:108200005554433A20253034642D253032642D25D1
:108210003032642020200000253032643A2530328C
:10822000643A2530326400007A372D6C6F672E7403
:10823000787400004572726F72206F70656E696E9F
:1082400067206C6F672066696C6520666F722077A7
:10825000726974653A2025640D0A00003D3D3D3D7C
:108260003D3D3D3D3D3D3D3D3D3D3D3D3D3D3D3D3E
:108270003D3D3D3D3D3D3D3D3D3D3D3D3D3D3D3D2E
:108280003D3D3D3D3D3D3D3D3D3D3D3D3D3D3D3D1E
:108290003D3D0D0A000000005A3720416C74696DA5
:1082A00065746572204D6F64756C650D0A00000081
:1082B00028632920323031352C204865787065726A
:1082C000742053797374656D730D0A0D0A000000F4
:1082D00056657273696F6E3A20322E32330D0A0082
:1082E0004275696C6420446174653A204D6179205F
:1082F000323320323031360D0A000000486172649A
:1083000077617265205265762025630D0A0D0A009B
:10831000203A20537461727475700D0A00000000D9
:10832000303A6C6F67253034642E6373760000003A
:10833000303A4C4F47253034642E6373760000008A
:10834000303A475053253034642E7478740000005E
:108350004572726F72206F70656E696E672064611E
:1083600074612066696C6520666F7220777269742B
:10837000653A2025640D0A00203A204F70656E652D
:108380006420646174612066696C652025732066D1
:108390006F722077726974650D0A0000203A204FD1
:1083A00070656E6564206770732066696C65202552
:1083B0007320666F722077726974650D0A00000081
:1083C000203A20436C6F7365642064617461206699
:1083D000696C650D0A000000203A20436C6F7365DC
:1083E00064206770732066696C650D0A00000000E8
:1083F000303A74657374312E747874004572726FFC
:1084000072206F70656E696E672066696C652066A4
:108410006F7220726561643A2025640A00000000D2
:1084200025730A00303A6C6F67303030302E747824
:10843000740000004572726F72206F70656E696E15
:10844000672066696C6520666F7220777269746553
:108450003A2025640A0000004F6E65206272696749
:108460006874206D6F726E696E672C20696E20745F
:108470006865206D6964646C65206F66207468654A
:10848000206E696768742C0A0000000074776F2002
:108490006465616420626F797320676F7420757002
:1084A00020746F2066696768742E20204261636BB8
:1084B00020746F206261636B0A0000007468657944
:1084C0002066616365642065616368206F74686518
:1084D000722C2064726577207468656972207377E6
:1084E0006F7264732C20616E640A000073686F748D
:1084F0002065616368206F746865722E20204120BA
:108500006465616620706F6C6963656D616E20687B
:108510006561726420746865206E6F6973652C0AEA
:1085200000000000616E642063616D6520616E640F
:10853000206B696C6C6564207468652074776F20AB
:108540006465616420626F79732E0A0A000000007E
:108550004E6F7720696620796F7520646F6E27747F
:108560002062656C69657665207468657365206C4A
:108570006965732061726520747275652C0A00004C
:1085800061736B2074686520626C696E64206D6134
:108590006E2E202048652073617720697420746FE7
:1085A0006F2E0A0028632920323031352C2048658F
:1085B00078706572742053797374656D730D0A0059
:1085C000253032643A253032643A253032640D0A5F
:1085D00000000000475053204669726D7761726554
:1085E0002056657273696F6E203A2025730D0A0D4F
:1085F0000A00000043256C753D256C75202573002D
:1086000044313D256C7525730000000044323D2542
:108610006C7525730000000044543D2564257300EB
:108620005A3D256425730000503D256C752E0000D1
:10863000256C75257300000025642E2530326400FA
:10864000545F696E743D25732573000025642E25E3
:1086500064000000545F6578743D25732573000045
:10866000484D3D256C642E0054696D652C20507278
:108670006573737572652C20545F496E7420256391
:108680002C20545F4578742025632C20416C74693C
:10869000747564652025632C2056696E2C20414436
:1086A000302C204144312C20414432002C205554A0
:1086B000432C204C61742C204E2F532C204C6F6E79
:1086C0002C20452F572C2053706565642025732C72
:1086D0002048656164696E672C2047505320416CC7
:1086E0007469747564652025632C2056616C696417
:1086F000000000002C2048756D696469747920259C
:1087000000000000496E6974204932430D0A0000E0
:10871000496E6974204C43440D0A00005A4C4F477F
:10872000205A37580000000056455220322E32336E
:108730000000000041444320496E697400000000BD
:10874000544D5020496E697400000000505A532067
:10875000496E697400000000465320496E69740038
:1087600043464720496E697400000000475053207B
:10877000496E6974000000004C4F4720496E6974CF
:1087800000000000202020475053204669726D777A
:108790006172652056657273696F6E203A20257389
:1087A0000D0A000052756E6E696E67005A202536FC
:1087B000640000004D20253664000000257320254C
:1087C0007300000050202534642E253032640000F0
:1087D0002530326468253032646D25303264000003
:1087E0005620202532642E2530336400484D202544
:1087F00032642E2530326425250000002534642E95
:1088000025326425630000002535642E253164255A
:108810006300000053202533642E253264000000DD
:1088200048202533642E253264000000475A25363F
:108830006400000025642C2025642E253032642C31
:108840002025732C2025732C2025642C2025642EB4
:10885000253033642C2025642E253033642C2025CC
:10886000642E253033642C2025642E253033642C6F
:108870002025642C2025642E253034642C2025638B
:108880002C2025642E253034642C2025632C2025B3
:10889000642E253034642C2025642E253034642C3D
:1088A0002025642C2025642C2025642E253032645C
:1088B0000000000025642C2025642E253032642C15
:1088C0002025732C2025732C2025642C2025642E34
:1088D000253033642C2025642E253033642C20254C
:1088E000642E253033642C2025642E253033642CEF
:1088F0002025642E25303264000000005CD4010085
:10890000031C00007119000051110000E803000071
:1089100047505320425244470000000020202020AE
:108920002020202000000000300D0A00310D0A0038
:10893000475053204669726D7761726520566572A3
:1089400073696F6E203D20004572726F72206F70E8
:10895000656E696E672066696C6520666F72207748
:10896000726974653A2025640D0A000025642C2084
:1089700025642E253034640D0A00000025640D0A9C
:10898000000000005357555044415445000000007A
:10899000CA5D00003E610000285E00003E610000EC
:1089A000EE5E00003E610000BA5F00003E61000024
:1089B000186000003E61000074600000202020204C
:1089C0002020202020202030202031202032202074
:1089D0003320203420203520203620203720203816
:1089E00020203920204120204220204320204420E4
:1089F00020452020460D0A00202020202020302065
:108A00002031202032202033202034202035202007
:108A100036202037202038202039202041202042B5
:108A20002020432020442020452020460D0A00001D
:108A30003031323334353637383941424344454694
:108A400000000000286E756C6C2900720077002A07
:108A50002A2A205F437379735F616C6C6F632066B1
:088A600061696C65640A00FF06
:108A6800F11FFF1F010001000B0000006D7068007E
:108A7800006B70680000000000010200090001009E
:108A8800DE07010139000000F6FFFFFF01000000CA
:108A980030F8FFFFC0D401006801000048E8010079
:108AA800BE010000C0D401002B02000038C1010043
:108AB800B4020000B0AD010064030000289A010070
:108AC80042040000A08601005C0500001873010044
:108AD800C2060000905F010088080000084C0100F1
:108AE800C90A000080380100AA0D0000F82401001E
:108AF80056110000701101002F120000880D0100AE
:108B080013130000A009010003140000B8050100B8
:108B1800FF140000D001010007160000E8FD000066
:108B28001D17000000FA00004118000018F60000A8
:108B38007219000030F20000B31A000048EE00007D
:108B4800041C000060EA0000651D000078E60000D3
:108B5800D71E000090E200005C200000A8DE0000A4
:108B6800F4210000C0DA0000A0230000D8D60000DD
:108B780061250000F0D200003827000008CF00006F
:108B88002629000020CB00002D2B000038C700004C
:108B98004D2D000050C30000882F000068BF000062
:108BA800DF31000080BB00005434000098B700009B
:108BB800E7360000B0B300009B390000C8AF0000E2
:108BC800713C0000E0AB00006B3F0000F8A700001C
:108BD8008B42000010A40000D145000028A000002E
:108BE80041490000409C0000DD4C000058980000FE
:108BF800A6500000709400009E5400008890000069
:108C0800C9580000A08C00005F5B0000488A000083
:108C1800225D0000B88800005F5F0000C486000085
:108C2800A7610000D0840000FA630000DC82000025
:108C380058660000E8800000C2680000F47E00006A
:108C4800386B0000007D0000BA6D00000C7B00004E
:108C58004870000018790000E272000024770000D4
:108C680089750000307500003C7800003C730000F6
:108C7800FD7A000048710000CA7D0000546F0000B2
:108C8800A4800000606D00008C8300006C6B000005
:108C980081860000786900008489000084670000EC
:108CA800948C000090650000B38F00009C63000066
:108CB800E0920000A86100001C960000B45F00006C
:108CC80067990000C05D0000C09C0000CC5B0000FC
:108CD80028A00000D8590000A0A30000E457000015
:108CE80027A70000F0550000BEAA0000FC530000B2
:108CF80065AE0000085200001CB2000014500000CD
:108D0800E3B50000204E0000BBB900002C4C000069
:108D1800A3BD0000384A00009DC10000444800007F
:108D2800A7C5000050460000C4C900005C4400000C
:108D3800F1CD00006842000031D20000744000000C
:108D480083D60000803E0000E7DA00008C3C00007B
:108D58005EDF0000983A0000E7E30000A438000056
:108D680083E80000B036000033ED0000BC3400009A
:108D7800F6F10000C8320000CDF60000D430000043
:108D8800B8FB0000E02E0000B8000100EC2C000049
:108D9800CB050100F82A0000F40A010004290000AC
:108DA8003110010010270000841501001C25000067
:108DB800EC1A0100282300006A2001003421000079
:108DC800FE250100401F0000A82B01004C1D0000DB
:108DD80069310100581B0000413701006419000087
:108DE8002F3D010070170000354301007C1500007D
:108DF8005349010088130000884F010094110000B6
:108E0800D6550100A00F000062580100D80E0000DE
:108E1800F35A0100100E0000875D0100480D0000A4
:108E28001F600100800C0000BB620100B80B00004D
:108E38005B650100F00A000000680100280A0000D4
:108E4800A86A010060090000546D0100980800003C
:108E580004700100D0070000B97201000807000083
:108E680072750100400600002E78010078050000A8
:108E7800EF7A0100B0040000B47D0100E8030000AF
:108E88007D800100200300004B8301005802000090
:108E98001C86010090010000EE880100C800000057
:108EA800CD8B010000000000A28E010038FFFFFFFB
:108EB8008691010070FEFFFF74940100A8FDFFFF7A
:108EC80058970100E0FCFFFF509A010018FCFFFFD3
:108ED8003E9D010050FBFFFF36A0010088FAFFFF0E
:108EE80038A30100C0F9FFFF00366E0100366E019D
:0400000300000115E3
:00000001FF
